:020000040800F2
:10000000305C0020E1010008494F0008693A00080F
:10001000C1460008010A0008B9600008000000009D
:10002000000000000000000000000000490100087E
:10003000FD0A0008000000008D010008815800083A
:10004000FB010008FB010008FB010008FB010008A0
:10005000FB010008FB010008FB010008FB01000890
:10006000FB010008FB010008FB010008FB01000880
:10007000FB010008A10A0008B10A0008C10A000833
:10008000FB010008FB010008D9070008FB0100087C
:10009000FB010008FB010008FB010008FB01000850
:1000A000FB010008FB010008FB010008FB01000840
:1000B0003559000851590008FB010008FB010008F0
:1000C000FB010008FB010008FB010008FB01000820
:1000D000FB01000815600008FB010008A96000088A
:1000E000FB010008FB010008FB010008FB01000800
:1000F000FB010008FB010008FB010008FB010008F0
:10010000FB010008FB010008FB010008FB010008DF
:10011000FB010008FB010008FB010008FB010008CF
:10012000FB010008FB010008FB010008FB010008BF
:10013000DFF810D000F004FB00480047F96A00081F
:10014000AFF30080305C0020224B19680868B0E8EB
:10015000F00F80F30988BFF36F8F4FF0000080F33A
:1001600011884EF00D0E7047000000000648006830
:10017000006880F3088862B661B6BFF34F8FBFF3A3
:100180006F8F00DF00BF00BF08ED00E0EFF30980D4
:10019000BFF36F8F0F4B1A6820E9F00F106008B59E
:1001A0004FF0500080F31188BFF34F8FBFF36F8F74
:1001B00007F008FD4FF0000080F31188BDE808400B
:1001C00019680868B0E8F00F80F30988BFF36F8FF3
:1001D000704700BFCC050020EFF30580704700009A
:1001E0000648804706480047FEE7FEE7FEE7FEE7D1
:1001F000FEE7FEE7FEE7FEE7FEE7FEE7335900080D
:1002000031010008202A04DB203A21FA02F0002103
:10021000704721FA02F3D040C2F120029140084316
:100220001946704740EA01039B0703D009E008C95B
:10023000121F08C0042AFAD203E011F8013B00F8AB
:10024000013B521EF9D27047D2B201E000F8012BF7
:10025000491EFBD270470022F6E710B513460A4646
:1002600004461946FFF7F0FF204610BD421C10F867
:10027000011B0029FBD1801A7047F0B480EA01020B
:10028000D40F4200B2EB410F02D20246084611469B
:100290004A0042D0C30DDDB2C1F3C752AD1A202DC2
:1002A00035DAC1F3160141F4000204B15242C5F13E
:1002B000200602FA06F12A411044B3EBD05F23D0A6
:1002C000C4B1012DA0EBC35009DCF0BC4FF00042DB
:1002D00002EAC352DBB200F5000000F0A6B940000C
:1002E00000F1807000EBC350A0F1807040EAD17043
:1002F000490009E0490841EAC071A0EBC35000F58C
:100300000000400800EBC350F0BC00F085B961422A
:10031000012202EB4101001BF6E7F0BC704781F0BF
:100320000041AAE780F00040A7E780EA010210B58B
:1003300002F00043400022D04A001FD0010E01EB22
:100340001261C0F35600C2F3560240F4000042F4BA
:100350000002A0FB022000047F39140400D0401CDE
:1003600050EA124001D44000491EC2B20C0604EB10
:10037000D010401C4008802A02D003E0002010BDAD
:1003800020F00100002900DA0020184310BD30B42D
:1003900080EA010202F0004530F0004221F0004006
:1003A00013D090B1C30DD40DC2F31601C0F31600E3
:1003B000E41A41F4000140F400027D34914201D37B
:1003C000641C00E04900002C02DA30BC00207047B9
:1003D0004FF400000023914201D3891A03434008DF
:1003E0004FEA4101F7D151B1914202D14FF00041A2
:1003F00005E002D24FF0010101E06FF0010103EBD3
:10040000C450284430BC00F007B92DE9FE4F81EA02
:10041000030404F0004421F0004100944FF0000B6D
:1004200023F0004350EA01045ED052EA03045BD09B
:10043000C3F30A54C1F30A552C44A4F2F3340194D3
:10044000A0FB0254C1F3130141F48011C3F3130361
:1004500043F4801301FB024400FB034E840A970A15
:1004600044EA815447EA8357A4FB076802958D0A42
:1004700005FB07854FEA932C04FB0C542705029DCE
:100480004FEA065847EA1637B5EB08056EEB070C3E
:10049000870E920E47EA811742EA8312A7FB0201F8
:1004A000B6EB0B0164EB00042B0D43EA0C335E1832
:1004B00044EB1C50DA465146E7FB0201C5F3130436
:1004C0004FEA0B3343EA14534FEA0432019C43EAE8
:1004D0000603A4F10C040294009CCDE900B400F0E2
:1004E000E1F803B0BDE8F08F00200146F9E7C10F45
:1004F00080EAE0700844CA079623002100F095B80E
:1005000096230022114600F090B820F00040C10D63
:10051000C0F3160040F400007F2901DA0020704784
:10052000962903DCC1F19601C8407047963988408E
:100530007047C1F30A5210B5C1F3130140F2FF3303
:1005400041F480119A4201DA002010BD40F2334399
:100550009A42A2F2334203DC5242FFF753FE10BD2F
:10056000904010BD00F0004230F000400AD0C10DB4
:1005700001F56071C0F3160042EA0151C20840075C
:100580001143704700200146704701F0004330B42A
:1005900021F0004150EA010206D00A0DA2F5607276
:1005A000C1F31301002A02DC30BC00207047440F65
:1005B00044EAC104C100E01830BC00EBC25000F0B6
:1005C0002BB80000002801DBC0F10040002901DB4E
:1005D000C1F1004181427047002801DBC0F10040B9
:1005E000002901DBC1F100418842704730B50B465C
:1005F000014600202022012409E021FA02F59D4253
:1006000005D303FA02F5491B04FA02F52844151E26
:10061000A2F10102F1DC30BD0029A8BF7047401CE7
:10062000490008BF20F00100704710B4B0FA80FC08
:1006300000FA0CF050EA010404BF10BC704749B145
:10064000CCF1200421FA04F411FA0CF118BF0121B5
:1006500021430843A3EB0C01CB1D4FEA00614FEA95
:10066000102042BF002010BC704700EBC350104464
:100670000029A4BF10BC7047401C490008BF20F0EF
:10068000010010BC704710B5141E73F1000408DAA5
:10069000401C41F1000192185B411A4301D120F046
:1006A000010010BD2DE9F04D92469B4611B1B1FA03
:1006B00081F202E0B0FA80F22032904600F052F867
:1006C00004460F4640EA0A0041EA0B0153465A46E7
:1006D000084313D0114653EA010019D0C8F1400273
:1006E0005046FFF78FFD05460E4650465946424696
:1006F00000F038F8084305D0012004E020463946D0
:10070000BDE8F08D0020054346EAE0762C433743F0
:100710000A986305E40AA0EB08000022FD0A44EAF7
:1007200047540A3002D500200146E9E701051019B7
:100730006941DDE9084500196941BDE8F04DA2E7CE
:10074000064C074D06E0E06840F0010394E807001E
:1007500098471034AC42F6D3FFF7EEFCC88100088E
:10076000E8810008202A04DB203A00FA02F1002088
:1007700070479140C2F1200320FA03F319439040DF
:10078000704770B58C1810F8015B15F0070301D1A4
:1007900010F8013B2A1106D110F8012B03E010F8E4
:1007A000016B01F8016B5B1EF9D12B0705D4002307
:1007B000521E0DD401F8013BFAE710F8013BCB1AA9
:1007C000921C03E013F8015B01F8015B521EF9D59E
:1007D000A142D8D3002070BD10B5024800F05FFCE4
:1007E00010BD0000800F002070B504460025206871
:1007F000806800F0010018B32068806820F00100D4
:100800002168886001F040FD054613E001F03CFDE1
:10081000401B02280ED92068806800F0010048B112
:10082000A06A40F01000A062E06A40F00100E062BF
:10083000012070BD2068806800F001000028E5D12B
:100840000020F6E738B50446002500200090206817
:10085000806800F0010078BB2068806840F00100EB
:1008600021688860194800681949B0FBF1F00090D0
:1008700002E00098401E009000980028F9D101F095
:1008800003FD054619E001F0FFFC401B022814D9C6
:100890002068806800F0010078B9A06A40F010007C
:1008A000A062E06A40F00100E06200BF002084F82E
:1008B000240000BF012038BD05E02068806800F0FA
:1008C00001000028DFD00020F5E70000C805002067
:1008D00040420F0010B5184806F002FD1749088085
:1008E000174806F0FDFC17490880144800884FF6A9
:1008F000FF71884202D01148008801E01248008848
:10090000114908800F4800884FF6FF71884202D0D5
:100910000C48008801E00D4800880C4908800A480E
:100920000088C0F30E000849088008480088C0F31A
:100930000E000649088010BD00180708900000202E
:100940000020070892000020A2000020A400002040
:10095000F0B597B006460D4601A803F0B5F800249F
:1009600012E004F50070854202D94FF4007700E0F0
:100970002F1B31193A461148FFF754FC3A460F49EC
:1009800001A803F0A1FC3C44AC42EAD301A90C4805
:1009900003F06CF8002407E00948005D0949615C38
:1009A000884200D002E0641C102CF5D300BF102C4C
:1009B00002D3012017B0F0BD0020FBE7002000208B
:1009C0001E28002000500708F0B50446187822F8C9
:1009D00010400025002004E032F810603544461C29
:1009E000F0B20A28F8DB0A20B5FBF0F0088018788E
:1009F000401C0A2690FBF6F706FB17001870F0BDA6
:100A000000BFFEE72DE9FC4707460D463846FFF7D5
:100A100077FD81462946FFF788FC04464FF08B415D
:100A2000FFF7B5FC064631462846FFF778FC8146BD
:100A300049463046FFF7ABFC04461549FFF775FC05
:100A40008046002419E0134A601C52F820104046EA
:100A5000FFF7C2FD10D80F4850F824104046FFF7AA
:100A6000B1FD09D20A2023460A4A0B49CDE90040CC
:100A7000404605F09BFE04E0641C40F2472084429F
:100A8000E1D300BF05480088FFF73AFDBDE8FC87C9
:100A900000002041F0020020A80000203C050020BA
:100AA00010B5024800F0F2FE10BD00009048002092
:100AB00010B5024800F0EAFE10BD00004C480020CE
:100AC00010B5024800F0E2FE10BD0000084800200A
:100AD00030B590F840500124AC40C56B6C600468A0
:100AE00063604468102C04D10468A2600468E1606B
:100AF00003E00468A1600468E26030BD704770B52F
:100B000003460024002010E00E5C451C4D5D46EAC3
:100B10000526851C4D5D46EA0546C51C4D5D46EA29
:100B2000056543F82450641C001D9042ECD370BD51
:100B300070B5034614460022002015E011F822503B
:100B40001D5431F82250C5F30726451C5E5551F857
:100B50002250C5F30746851C5E5551F822502D0ED4
:100B6000C61C9D55521C001DA042E7D370BD72B635
:100B700000BFFEE70021074AD1610749096941F03A
:100B80000401054A11611146096941F040011161F2
:100B90007047000020490020002002400021074A41
:100BA000D1610749096941F00201054A1161114605
:100BB0004861096941F040011161704720490020F6
:100BC000002002400022054BDA61054A126942F01A
:100BD0000102034B1A610180704700002049002088
:100BE0000020024000201E49C96801F0100139B1FF
:100BF0001C49C96941F002011A4AD16140F0100054
:100C00001749C96801F0040139B11649C96941F0B1
:100C10000101144AD16140F004001149C96901F091
:100C2000010169B10F49C96941F004010D4AD1615F
:100C300000BF0B49C96921F00101094AD16100BF18
:100C400000BF40F20111884206D10549C96921F06F
:100C50000101034AD16101E00149C86000BF70474A
:100C6000002002402049002070B5044601F00CFB32
:100C7000054609E0601C38B124B101F005FB401BBA
:100C8000A04201D9032070BD1248C06800F00100E5
:100C90000028EFD10F48C06800F0200020B100BF4D
:100CA00020200C49C86000BF0A48C06800F010004E
:100CB00048B90848C06900F0010020B90548C0687B
:100CC00000F0040018B1FFF78DFF0120DBE70020E2
:100CD000D9E7000000200240F0B503461C4600257D
:100CE0000026084607E010F8015B10F8016B45EAA2
:100CF000062724F8027B171EA2F1010C1FFA8CF2C2
:100D0000F1D1F0BD2DE9F04786B080460E46914600
:100D10004FF0000A00270025C6F30A0AA6EB0A07CF
:100D2000002005900190039701200490820239462B
:100D30001548FFF7D1FF00BF07E038F8150005EBB5
:100D40005A01114A22F811006D1C4D45F5D301F0EE
:100D5000CBF805A901A801F00DF800240BE00A4822
:100D600030F814C007EB440162460023012001F073
:100D700063F8601C84B2B4F5806FF0DB01F052F8C8
:100D800006B0BDE8F0870000001000202DE9F04714
:100D900081463A4800F0BEFB6421384800F0FAFA78
:100DA000364800F078F986B235493046FFF72AFE1A
:100DB0008046FFF7AAFB87B2324B334A33493846A5
:100DC000FFF702FE2D4800F0A5FB64212B4800F040
:100DD000E1FA2A4800F05FF985B22D480580B5B1E7
:100DE0002C48008800F4004010B12B48008802E035
:100DF000294800884042284485B240F68B60274944
:100E0000088008460088854201DB08460588244B97
:100E1000244A25492846FFF7D7FD184800F07AFBF9
:100E20006421164800F0B6FA144800F034F984B290
:100E30001E480480B4B11E48008800F4004010B180
:100E40001C48008802E01B4800884042204484B2CD
:100E500040F68B601849088008460088844201DB10
:100E600008460488154B164A16492046FFF7ACFD84
:100E7000024800F0E7FBBDE8F0870000800F00208B
:100E8000333353409A000020B00F0020940000201C
:100E90009E00002090000020A200002038050020C5
:100EA0009B000020C40F002096000020A00000201E
:100EB00092000020A40000203A0500209C000020A1
:100EC000D80F0020980000202DE9F04100250024D3
:100ED0001EE0002600270CE0104A02EBC4029188B5
:100EE0000E4A52F8340004F043FB304486B2781CBA
:100EF000C7B20A2FF0DB052E04DB0120A0402843F7
:100F0000C5B203E00020A0402843C5B2601CC4B2B3
:100F1000082CDEDB2846BDE8F0810000B080000828
:100F200002490968C1F3C300704700000C0C01407E
:100F30007047000038B5024600230020009000BF33
:100F400092F82400012801D1022038BD012082F846
:100F5000240000BF4868072812D21068406B0C7943
:100F6000641E04EB84051F24AC40A0430D796D1E64
:100F700005EB85050C68AC4020431468606327E0EE
:100F800048680D2812D21068006B0C79E41F04EB3E
:100F900084051F24AC40A0430D79ED1F05EB8505AA
:100FA0000C68AC4020431468206311E01068C06AEC
:100FB0000C790D3C04EB84051F24AC40A0430D7953
:100FC0000D3D05EB85050C68AC4020431468E062DC
:100FD00008680A2812D31068C0680C780A3C04EB31
:100FE00044050724AC40A0430D780A3D05EB4505B8
:100FF0008C68AC4020431468E0600FE01068006922
:101000000C7804EB44050724AC40A0430D7805EBB5
:1010100045058C68AC40204314682061086810289E
:1010200002D00868112827D1174C1068A0421ED1A1
:101030001068806800F40000F0B91068806840F41F
:1010400000001468A0600868102815D10F480068D7
:101050000F4CB0FBF4F000EB80004000009002E089
:101060000098401E009000980028F9D104E0906A92
:1010700040F020009062012300BF002082F824008D
:1010800000BF184661E7000000240140C8050020A9
:1010900040420F00704701460868C06C704770B549
:1010A0000446206805682068466806F0200020286D
:1010B0002DD105F00200022829D1A06A00F010000D
:1010C00018B9A06A40F40070A0622068806800F43B
:1010D0006020B0F5602F13D1207B88B9206840686C
:1010E00020F0200021684860A06A20F48070A0628F
:1010F000A06A00F4805018B9A06A40F00100A06214
:101100002046FFF7C7FF6FF012002168086006F065
:101110008000802839D105F00400042835D1A06A68
:1011200000F0100018B9A06A40F40050A0622068D6
:10113000806800F4E040B0F5E04F0DD020684068D2
:1011400000F48060D0B92068806800F46020B0F5B9
:10115000602F13D1207B88B92068406820F0800080
:1011600021684860A06A20F48050A062A06A00F460
:10117000807018B9A06A40F00100A0622046FFF715
:10118000D7FE6FF00C002168086006F04000402890
:101190000DD105F0010050B1A06A40F48030A0628A
:1011A000204600F0B5F86FF001002168086070BDBE
:1011B0002DE9F0410446002700250026A84614B971
:1011C0000120BDE8F081A06810B1207D00B100BF12
:1011D000A06A30B90020E06284F82400204600F0C4
:1011E00099F82046FFF700FB0746A06A00F01000C0
:1011F000002873D1002F7ED1A06A20F4885040F0DF
:101200000200A0623F4AD4E90001904208D1E0699F
:10121000B0F5402F02D14FF4002002E0E06900E079
:10122000E0690143207B41EA40000643A068B0F535
:10123000807F02D0A068012802D14FF4807000E0C6
:1012400000200543207D012811D1207B38B9A069F9
:10125000401E4FF4006141EA4030054307E0A06AB8
:1012600040F02000A062E06A40F00100E0622068E7
:10127000406820F4694028432168486020688068FD
:1012800021490840304321688860A068B0F5807F1C
:1012900002D0A068012802D14FF4807000E0002045
:1012A000B0F5807F03D1208A401E4FEA00582068A5
:1012B000C06A20F4700040EA08002168C862206813
:1012C000806812490840B04209D10020E062A06A5B
:1012D00020F0020040F00100A06211E00BE0A06AE3
:1012E00020F0020040F01000A062E06A40F001002F
:1012F000E062012704E0A06A40F01000A06201272C
:1013000038465EE7003C0140FDF7E1FFFE0E1FFF9F
:101310007047000010B586B004460020029003908C
:10132000049005901849206888422AD100BF1748C8
:10133000806940F40070154988610846806900F4AE
:101340000070019000BF00BF00BF0846806940F0F8
:10135000100088610846806900F01000019000BF0D
:1013600000BF072002900320039002A9084800F064
:10137000D3FD00220521122001F046F8122001F0D1
:1013800033F806B010BD00000024014000100240F8
:1013900000100140F8B504460D46002600200090DC
:1013A000002700F071FF06462068806800F4807016
:1013B00050B1A06A40F02000A06200BF002084F875
:1013C000240000BF0120F8BD2068406800F4807050
:1013D00020BB2068C06A00F47000F8B917E0681CF0
:1013E000A8B125B100F050FF801BA8420FD920689A
:1013F000006800F0020050B9A06A40F00400A0624A
:1014000000BF002084F8240000BF0320DBE7206831
:10141000006800F002000028E1D053E0022001F053
:1014200067F838490968B1FBF0F021680969364A64
:10143000114091B92168C9689211114069B92168B8
:101440000969324A114031B92168C96892111140C5
:1014500009B9142117E0292115E0216809692B4AEF
:10146000114021B92168C9689211114041B1216828
:101470000969274A114029B92168C968114009B989
:10148000542100E0FC2100FB01F718E0681C98B132
:1014900025B100F0F9FE801BA8420DD90098B84292
:1014A0000AD2A06A40F00400A06200BF002084F8C5
:1014B000240000BF032086E70098401C009000989D
:1014C000B842E3D36FF0120021680860A06A40F4CC
:1014D0000070A0622068806800F46020B0F5602F82
:1014E0000DD1207B58B9A06A20F48070A062A06A58
:1014F00000F4805018B9A06A40F00100A0620020FA
:1015000061E70000C8050020244992249224491272
:101510004992240070B50446002500BF94F82400C9
:10152000012801D1022070BD012084F8240000BFF1
:101530002046FFF787F90546002D77D1A06A40F2D3
:101540000121884340F48070A0623C4920688842B1
:1015500008D13B48006800F4702008B9012002E07F
:10156000002000E0012078B1A06A20F48010A06281
:101570002068406800F4806000B3A06A20F4005046
:1015800040F48050A06219E0A06A40F48010A0628C
:101590002B49091F2068884203D0284920688842C7
:1015A00004D12748006800F4806000E0002028B1E2
:1015B000A06A20F4005040F48050A062A06A00F4B9
:1015C000805020B1E06A20F00600E06201E00020D7
:1015D000E06200BF002084F8240000BFC01E216824
:1015E00008602068806800F46020B0F5602F16D194
:1015F00012492068884208D11148006800F4702020
:1016000008B9012002E0002000E0012038B1206884
:10161000806840F4A000216888600CE006E0206843
:10162000806840F480102168886004E000BF0020DA
:1016300084F8240000BF284675E700000028014018
:101640000424014070B50446002500BF94F824002E
:10165000012801D1022070BD012084F8240000BFC0
:101660002046FFF7C1F805462DB9A06A20F488503E
:1016700040F00100A06200BF002084F8240000BFF9
:101680002846E8E70146002291F82100022808D008
:101690000420886300BF002081F8200000BF0120E3
:1016A00070470868006820F00E000B681860086832
:1016B000006820F001000B68186091F840300120AC
:1016C0009840CB6B5860012081F8210000BF0020BA
:1016D00081F8200000BF1046E2E7000070B5044624
:1016E000002594F82100022803D00420A0630125DE
:1016F000C1E02068006820F00E00216808602068C2
:10170000006820F00100216808605C492068884278
:1017100052D95A4978392068884201D1012047E0DE
:10172000564964392068884201D1102040E053496D
:1017300050392068884201D1801539E04F493C3941
:101740002068884201D1801432E04C492839206851
:10175000884202D14FF480302AE048491439206889
:10176000884202D14FF4801022E044492068884228
:1017700001D140041CE042492068884201D1012087
:1017800016E03F4914312068884201D110200FE053
:101790003B4928312068884201D1801508E038494A
:1017A0003C312068884201D1801401E04FF4803040
:1017B0003349091F086051E0304978392068884270
:1017C00001D1012047E02D4964392068884201D1C8
:1017D000102040E0294950392068884201D1801505
:1017E00039E026493C392068884201D1801432E032
:1017F000224928392068884202D14FF480302AE0FB
:101800001E4914392068884202D14FF4801022E02A
:101810001A492068884201D140041CE01849206818
:10182000884201D1012016E0154914312068884210
:1018300001D110200FE0124928312068884201D1DF
:10184000801508E00E493C312068884201D180149F
:1018500001E04FF48030094980394860012084F864
:10186000210000BF002084F8200000BF606B10B191
:101870002046616B8847284670BD0000800002400A
:10188000080402400146886B7047000070B50446AA
:10189000E06B05682068066894F8401004208840D2
:1018A0002840002875D006F004000028FAD02068EF
:1018B000006800F0200028B92068006820F00400CB
:1018C00021680860D5492068884254D9D3497839BD
:1018D0002068884201D1042049E0D0496439206859
:1018E000884201D1402042E0CC49503920688842EA
:1018F00001D100153BE0C9493C392068884202D13A
:101900004FF4804033E0C54928392068884202D12D
:101910004FF480202BE0C14914392068884202D15D
:101920004FF4800023E0BD492068884201D1C00403
:101930001DE0BB492068884201D1042017E0B84966
:1019400014312068884201D1402010E0B449283188
:101950002068884201D1001509E0B1493C31206876
:10196000884202D14FF4804001E04FF48020AC491E
:10197000091F086054E0A94978392068884201D1DC
:1019800004204AE0A54964392068884202D14020F9
:1019900043E04CE0A14950392068884201D100154C
:1019A0003BE09E493C392068884202D14FF4804098
:1019B00033E09A4928392068884202D14FF48020C8
:1019C0002BE0964914392068884202D14FF48000F8
:1019D00023E092492068884201D1C0041DE090496B
:1019E0002068884201D1042017E08D491431206815
:1019F000884201D1402010E089492831206888427E
:101A000001D1001509E086493C312068884202D1A5
:101A10004FF4804001E04FF48020804980394860D5
:101A2000E06A002802D02046E16A8847F4E094F892
:101A30004010022088402840002871D006F00200A3
:101A40000028FAD02068006800F0200040B9206823
:101A5000006820F00A0021680860012084F8210055
:101A60006E492068884254D96C4978392068884288
:101A700001D1022049E0694964392068884201D1D6
:101A8000202042E0654950392068884201D1401544
:101A90003BE062493C392068884202D14FF4005053
:101AA00033E05E4928392068884202D14FF4003083
:101AB0002BE05A4914392068884202D14FF40010B3
:101AC00023E056492068884201D180041DE0544932
:101AD0002068884201D1022017E051491431206862
:101AE000884201D1202010E04D49283120688842E9
:101AF00001D1401509E04A493C312068884202D1B1
:101B00004FF4005001E04FF400304549091F0860D0
:101B100054E0424978392068884202D102204AE0E4
:101B200057E03E4964392068884201D1202042E0D4
:101B30003A4950392068884201D140153BE0374985
:101B40003C392068884202D14FF4005033E03349D9
:101B500028392068884202D14FF400302BE02F4909
:101B600014392068884202D14FF4001023E02B4939
:101B70002068884201D180041DE0294920688842FC
:101B800001D1022017E0264914312068884201D192
:101B9000202010E0224928312068884201D14015D8
:101BA00009E01F493C312068884202D14FF40050BF
:101BB00001E04FF4003019498039486000BF00202F
:101BC00084F8200000BFA06A30B32046A16A88478D
:101BD00022E094F84010082088402840E0B106F048
:101BE0000800C8B12068006820F00E002168086075
:101BF00094F8401001208840E16B48600120A06308
:101C000084F8210000BF002084F8200000BF206B72
:101C100010B12046216B884770BD00008000024053
:101C2000080402400146002209B9012070471E4BFA
:101C3000086898420BD21D4B0868C01A1423B0FBE9
:101C4000F3F08000086419480838C8630AE0164BAE
:101C50000868C01A1423B0FBF3F08000086412482F
:101C60000838C863022081F821000868026843F63A
:101C7000F0708243D1E901031843CB6818430B6924
:101C800018434B6918438B691843CB6918430243C7
:101C90000868026000208863012081F8210000208C
:101CA00081F8200000BFC1E708040240080002409C
:101CB0002DE9F04104460D4616461F464FF0000838
:101CC00000BF94F82000012802D10220BDE8F08175
:101CD000012084F8200000BF94F8210001282CD1B5
:101CE000022084F821000020A0632068006820F012
:101CF0000100216808603B46324629462046FEF72F
:101D0000E7FEE06A30B12068006840F00E0021680C
:101D100008600BE02068006820F00400216808607B
:101D20002068006840F00A002168086020680068A8
:101D300040F001002168086006E000BF002084F840
:101D4000200000BF4FF002084046BFE770B50446D0
:101D500000F09AFA06462546681C10B1044800783F
:101D6000054400BF00F090FA801BA842FAD370BD72
:101D7000C40500202DE9F04104460E460127002548
:101D800000BF2648007E012802D10220BDE8F08174
:101D900001202249087600BF2068022813D14CF2A6
:101DA0005030FEF761FF90BB0120FEF7E3FE4CF2DE
:101DB0005030FEF759FF07461948006920F004002B
:101DC0001749086123E04CF25030FEF74DFFF0B99F
:101DD0004FF0FF303060A56812E02846FEF7DEFEC7
:101DE0004CF25030FEF740FF07460D48006920F0E6
:101DF00002000B4908610FB1356007E005F5006589
:101E0000D4E9021001EBC020A842E6D800BF00BF11
:101E100000200249087600BF3846B7E72049002075
:101E2000002002400348006940F080000149086139
:101E300000207047002002402DE9FE4F05468B46EA
:101E400017469846012600240020029000BF24482F
:101E5000007E012802D10220BDE8FE8F012020492A
:101E6000087600BF4CF25030FEF7FEFE064686BBF9
:101E7000012D02D10120029006E0022D02D10220A4
:101E8000029001E00420029000241EE02201B946E5
:101E9000C24648465146FEF7B5F980B2019002208D
:101EA00000FB04B000900199FEF78CFE4CF250301C
:101EB000FEF7DAFE06460B48006920F001000949EA
:101EC000086106B104E0601CC4B202988442DDDB04
:101ED00000BF00BF00200249087600BF3046BBE7C4
:101EE000204900200020024000200849096901F033
:101EF000800151B10649054A5160064951601146B9
:101F0000096901F0800101B1012070470020024001
:101F100023016745AB89EFCD2DE9F8470246002341
:101F20009C467BE14FF0010808FA03F4D1F80080E9
:101F300008EA0400A0427DD1DFF8F4A2D1F80480C1
:101F4000A8EB0A09D0453AD014DCB8F1030F50D001
:101F500009DCB8F1000F31D0B8F1010F1CD0B8F195
:101F6000020F49D120E0B8F1110F18D0B8F1120FCB
:101F700042D11EE0B9F5881F25D006DCB9F5803FB7
:101F800020D0B9F5801F37D11AE0B9F5001F18D05D
:101F9000B9F5041F30D117E0D1F80CC02DE0D1F80D
:101FA0000C8008F1040C28E0D1F80C8008F1080C32
:101FB00023E0D1F80C8008F10C0C1EE000BF00BF3C
:101FC00000BF00BF00BF00BFD1F80880B8F1000F0C
:101FD00002D14FF0040C0BE0D1F80880B8F1010FEA
:101FE00003D14FF0080C146102E04FF0080C54616B
:101FF00003E04FF0000C00E000BF00BFFF2801D855
:10200000904601E002F104084646FF2802D84FEA54
:10201000830803E0A3F108084FEA88084746D6F88A
:1020200000804FF00F0909FA07F928EA09080CFAAD
:1020300007F900E07AE048EA0908C6F80080D1F81C
:10204000048008F08058B8F1805F6FD100BFDFF8DE
:10205000E481D8F8188048F00108DFF8D891C9F871
:102060001880C846D8F8188008F00108CDF800801C
:1020700000BF00BF4FEAB9384FEA930958F829501A
:102080004FEA83784FEA18794FF00F0808FA09F8F9
:1020900025EA0805DFF8A081424502D14FF000088B
:1020A00024E0DFF89881424502D14FF001081DE09D
:1020B000DFF88C81424502D14FF0020816E0DFF8CC
:1020C0008481424502D14FF003080FE0DFF87881A8
:1020D000424502D14FF0040808E0DFF87081424524
:1020E00002D14FF0050801E04FF006084FEA83796E
:1020F0004FEA197908FA09F848EA0505DFF850812E
:102100004FEA930948F82950D1F8048008F4801860
:10211000B8F5801F0BD1DFF83C81D8F8008048EA81
:102120000008DFF83091C9F800800AE075E0DFF8B8
:102130002481D8F8008028EA0008DFF81891C9F84F
:102140000080D1F8048008F40018B8F5001F0ED103
:10215000DFF8008108F10408D8F8008048EA000898
:10216000DFF8F09009F10409C9F800800DE0DFF80C
:10217000E48008F10408D8F8008028EA0008DFF8B5
:10218000D49009F10409C9F80080D1F8048008F45A
:102190000038B8F5003F0ED1DFF8B880A8F1040888
:1021A000D8F8008048EA0008DFF8A890A9F10409EF
:1021B000C9F800800DE0DFF89C80A8F10408D8F889
:1021C000008028EA0008DFF88C90A9F10409C9F81A
:1021D0000080D1F8048008F48038B8F5803F0ED133
:1021E000DFF87080A8F10808D8F8008048EA0008F5
:1021F000DFF86090A9F10809C9F800800DE0DFF868
:102200005480A8F10808D8F8008028EA0008DFF810
:102210004490A9F10809C9F800805B1CD1F800803E
:1022200028FA03F8B8F1000F7FF47CAEBDE8F88718
:10223000000011100010024000080140000C014095
:10224000001001400014014000180140001C014032
:102250000800014008040140024693680B400BB19E
:10226000012000E00020704710B5C26821EA020397
:1022700002EA010443EA0443036110BD0AB10161AB
:1022800001E00B04036170470148006870470000DB
:10229000BC05002003480068034909780844014947
:1022A00008607047BC050020C405002010B5084830
:1022B000006840F0100006490860032000F0E2F8D2
:1022C0000F2000F007F800F05FF8002010BD0000BC
:1022D000002002402DE9F04188B004460027B846AE
:1022E000002600BF2348C06940F002002149C861B0
:1022F0000846C06900F00200019000BF00BF02A9BB
:1023000003A800F0DFFA069F1FB900F003FB0546A3
:1023100002E000F0FFFA45001748B5FBF0F0A0F12D
:10232000010816481649086040F2E7311448C160B8
:10233000C0F80480002101618160816100F0C4FD6A
:10234000064696B90E4800F013FE06466EB91D20EB
:1023500000F04AF8102C07D2002221461D2000F080
:1023600053F80848046000E00126304608B0BDE894
:10237000F08100000010024040420F0000040040C5
:10238000D4480020C005002008B500BF144880696B
:1023900040F00100124988610846806900F00100A0
:1023A000009000BF00BF00BF0846C06940F08050E9
:1023B000C8610846C06900F08050009000BF00BFAF
:1023C00000220F21901E00F01FF800BF0549486849
:1023D00020F0E06040F00070486000BF08BD0000E1
:1023E000001002400000014001460846002809DBB9
:1023F00000F01F0301229A4043099B0003F1E023F0
:10240000C3F8002100BF70472DE9F05F80460D46FC
:102410001646002703F010FF074639462A46334682
:1024200001F00700C0F1070ABAF1040F02D94FF01A
:10243000040A01E0C0F1070AD14600F1040ABAF12A
:10244000070F02D24FF0000A01E0A0F1030AD446C0
:102450004FF0010A0AFA09FAAAF1010A0AEA020A85
:102460000AFA0CFA4FF0010B0BFA0CFBABF1010B63
:102470000BEA030B4AEA0B042146404603F0E4FE54
:10248000BDE8F09F00BF00F00702064B19684FF649
:10249000FF031940044B0B4343EA0221014B19602F
:1024A00000BF70470CED00E00000FA0500BF00BF60
:1024B00000BF00BF00BFBFF34F8F00BF00BF00BF12
:1024C0000948006800F4E06008490843001D064917
:1024D000086000BF00BF00BFBFF34F8F00BF00BF49
:1024E00000BF00BF00BFFDE70CED00E00000FA05F3
:1024F0002DE9F04706464FF000080025002700248C
:10250000A146042E37D004DC012E3CD0022E6CD123
:1025100060E0082E33D0102E67D13648446800683A
:1025200000F0807008B33448C4F38341475C04F47E
:10253000803078B12F484068C0F340402F4911F8EF
:10254000008004F4803040B12D48B0FBF8F000FB6F
:1025500007F502E02B4807FB00F52648406800F429
:102560008000B0F5800F01D1A94603E06800032187
:10257000B0FBF1F93AE000F0EDF9814636E000F009
:10258000E9F9814632E01B48046A04F44070B0F572
:10259000807F05D104F0020010B14FF4004918E02B
:1025A00004F44070B0F5007F07D11248406A00F093
:1025B000020010B149F640490BE004F44070B0F558
:1025C000407F06D10B48006800F4003008B14FF29C
:1025D00024490BE000F0AEF906494968C1F38131A6
:1025E000491C4900B0FBF1F900E000BF00BF4846BC
:1025F000BDE8F08700100240728100088281000867
:1026000000127A0000093D00F8B5044600260025B6
:10261000207800F0010000286BD000274348C069F3
:1026200000F0805070B900BF4048C06940F0805051
:102630003E49C8610846C06900F08050009000BF64
:1026400000BF01273A48006800F48070B0B93848EC
:10265000006840F4807036490860FFF715FE0646B2
:1026600006E0FFF711FE801B642801D90320F8BDA6
:102670002F48006800F480700028F2D02B48006AD0
:1026800000F440752DB3A08800F44070A84220D01B
:102690002648006A20F44075012026490860002081
:1026A00008602248056205F0010090B1FFF7ECFDDB
:1026B000064608E0FFF7E8FD801B41F288318842BA
:1026C00001D90320D3E71948006A00F0020000286E
:1026D000F0D01648006A20F440706168084313493E
:1026E0000862012F04D10846C06920F08050C861FB
:1026F00000BF207800F00200022807D10B48406894
:1027000020F44040A168084308494860207800F060
:102710001000102807D10548406820F48000616946
:102720000843024948600020A1E700000010024071
:10273000007000404004424270B504460D460CB99A
:10274000012070BD5A48006800F00700A8420ED270
:102750005748006820F0070028435549086008469C
:10276000006800F00700A84201D00120E9E72078C6
:1027700000F0020002281DD1207800F00400042897
:1027800005D14C48406840F4E0604A4948602078F0
:1027900000F00800082805D14648406840F4605021
:1027A000444948604348406820F0F000A16808436D
:1027B00040494860207800F0010078B36068012843
:1027C00006D13C48006800F4003090B90120B8E719
:1027D0006068022806D13748006800F0007040B9F0
:1027E0000120AEE73348006800F0020008B901207C
:1027F000A7E73048406820F00300616808432D498E
:102800004860FFF741FD064609E0FFF73DFD801BEC
:1028100041F28831884202D9032092E707E0254837
:10282000406800F00C006168B0EB810FEDD12048EA
:10283000006800F00700A8420ED91D48006820F08B
:10284000070028431A4908600846006800F007009E
:10285000A84201D0012074E7207800F00400042889
:1028600007D11448406820F4E060E168084311494A
:102870004860207800F00800082808D10D4840681A
:1028800020F46050216940EAC1000A49486000F024
:1028900061F808494968C1F30311074A515CC8400F
:1028A0000649086006480068FFF714FD002048E765
:1028B000002002400010024084810008C80500206A
:1028C000C00500200F2202600D4A526802F0030288
:1028D00042600B4A526802F0F0028260084A526875
:1028E00002F4E062C260064A526802F46052D20802
:1028F0000261044A126802F007020A607047000091
:1029000000100240002002400148006870470000AB
:10291000C805002000B5FFF7F7FF04494968C1F377
:102920000221034A515CC84000BD00000010024073
:102930009481000800B5FFF7E7FF04494968C1F337
:10294000C221034A515CC84000BD00000010024093
:102950009481000870B5002100220024002300208B
:10296000134D696801F00C05F5B1042D02D0082D56
:1029700019D101E00F4819E00F4DC1F38346AB5D5B
:1029800001F4803555B10A4D6D68C5F340450B4ED5
:10299000725D084D5D43B5FBF2F402E0084D03FBA8
:1029A00005F4204602E000BF024800BF00BF70BD32
:1029B0000010024000127A00608100087081000857
:1029C00000093D00F8B504460CB90120F8BD207897
:1029D00000F00100002878D0F848406800F00C00B2
:1029E00004280CD0F548406800F00C00082811D1EC
:1029F000F248406800F48030B0F5803F0AD1EF48DB
:102A0000006800F4003000285FD0606800285CD1C6
:102A10000120DBE700BF6068B0F5803F06D1E748E2
:102A2000006840F48030E549086028E0606858B9E3
:102A3000E248006820F48030E049086008460068F9
:102A400020F4802008601AE06068B0F5A02F0BD158
:102A5000DA48006840F48020D849086008460068D9
:102A600040F4803008600AE0D448006820F48030E8
:102A7000D24908600846006820F48020086000BF42
:102A8000606888B1FFF700FC054606E0FFF7FCFB35
:102A9000401B642801D9032098E7C848006800F467
:102AA00000300028F2D010E0FFF7EEFB054606E00C
:102AB000FFF7EAFB401B642801D9032086E7BF48E3
:102AC000006800F400300028F2D1207800F0020005
:102AD000022857D1B948406800F00C0050B1B748FF
:102AE000406800F00C00082818D1B448406800F491
:102AF000803098B9B148006800F0020020B1206928
:102B0000012801D0012061E7AC48006820F0F800FE
:102B1000616940EAC100A949086033E02069E8B171
:102B20000120A7490860FFF7AFFB054606E0FFF765
:102B3000ABFB401B022801D9032047E79F480068F0
:102B400000F002000028F2D09C48006820F0F80055
:102B5000616940EAC1009949086013E00020984982
:102B60000860FFF791FB054606E0FFF78DFB401B71
:102B7000022801D9032029E79048006800F00200EC
:102B80000028F2D1207800F0080008282DD1A06993
:102B9000B8B101208B490860FFF776FB054606E0D7
:102BA000FFF772FB401B022801D903200EE7834880
:102BB000406A00F002000028F2D0012002F0C4FCBC
:102BC00013E000207F490860FFF75EFB054606E042
:102BD000FFF75AFB401B022801D90320F6E677488D
:102BE000406A00F002000028F2D1207800F00400D2
:102BF000042873D100277148C06900F0805070B973
:102C000000BF6E48C06940F080506C49C8610846FA
:102C1000C06900F08050009000BF00BF01276A48E3
:102C2000006800F48070B0B96748006840F48070B4
:102C300065490860FFF728FB054606E0FFF724FB1F
:102C4000401B642801D90320C0E65F48006800F4F7
:102C500080700028F2D000BFE068012806D15748F4
:102C6000006A40F001005549086227E0E06858B961
:102C70005248006A20F00100504908620846006A84
:102C800020F00400086219E0E06805280BD14B48E9
:102C9000006A40F00400494908620846006A40F0B2
:102CA000010008620AE04548006A20F0010043493B
:102CB00008620846006A20F00400086200BFE0686D
:102CC000A0B1FFF7E1FA054609E0FFF7DDFA401B86
:102CD00041F28831884202D9032077E622E0374862
:102CE000006A00F002000028EFD012E0FFF7CCFAF3
:102CF000054608E0FFF7C8FA401B41F288318842D8
:102D000001D9032062E62D48006A00F00200002885
:102D1000F0D1012F05D12948C06920F08050274902
:102D2000C86100BFE069C8B32448406800F00C00E7
:102D3000082860D0E069022848D1002020490866B0
:102D4000FFF7A2FA054606E0FFF79EFA401B0228AD
:102D500001D903203AE61948006800F00070002805
:102D6000F2D1206AB0F5803F07D11448406820F4C2
:102D70000030A168084311494860D4E908010843BC
:102D80000E49496821F4741108430C494860012038
:102D90000B490866FFF778FA054607E03DE0FFF7C4
:102DA00073FA401B022801D903200FE6034800688C
:102DB00000F000700028F2D02FE000000010024068
:102DC000000042428004424200700040002014494A
:102DD0000866FFF759FA054606E0FFF755FA401B6B
:102DE000022801D90320F1E50E48006800F00070C8
:102DF0000028F2D111E0E069012800D1E6E5094898
:102E0000466806F48031206A814204D106F47011CC
:102E1000606A814201D00120D8E50020D6E500009B
:102E200000004242001002407047704730B5024631
:102E30000B4600BF92F83C00012801D1022030BDB2
:102E4000012082F83C0000BF022082F83D0010689B
:102E500044681068816824F070041868044310689E
:102E60004460144D1068A84213D0134D1068A84256
:102E70000FD01068B0F1804F0BD0104D1068A842F1
:102E800007D00F4D1068A84203D00E4D1068A8421D
:102E900005D121F08001586801431068816001204C
:102EA00082F83D0000BF002082F83C0000BF00BF58
:102EB000C5E70000002C0140003401400004004040
:102EC00000080040000C004010B504460CB9012079
:102ED00010BD94F83D0028B9002084F83C0020463D
:102EE00000F026F8022084F83D00211D206802F041
:102EF00037FD012084F8460000BF84F83E00012120
:102F00003F200155402001554120015500BF00BF21
:102F1000012084F8420043200155442001554520FA
:102F2000015500BF012084F83D000020D0E70000DB
:102F300038B504462068B0F1804F15D100BF0B486A
:102F4000C06940F001000949C8610846C06900F045
:102F50000100009000BF00BF002205211C20FFF7E8
:102F600053FA1C20FFF740FA38BD00000010024061
:102F7000014691F83D00012801D001207047022050
:102F800081F83D000868C06840F001000B68D86017
:102F9000164B0868984213D0154B086898420FD01A
:102FA0000868B0F1804F0BD0124B0868984207D0E8
:102FB000114B0868984203D0104B086898420CD116
:102FC0000868806800F00702062A0CD008680068CC
:102FD00040F001000B68186005E00868006840F0E8
:102FE00001000B6818600020C8E70000002C0140B9
:102FF000003401400004004000080040000C004084
:103000002DE9F04104460D46002700BF94F83C002E
:10301000012802D10220BDE8F081012084F83C00A3
:1030200000BF022084F83D002068866826F07706FD
:1030300026F47F46206886602868502833D00CDC50
:10304000202850D004DC00284BD0102851D149E072
:10305000302849D040284CD139E060282DD0702844
:1030600007D0B0F5805F03D0B0F5005F41D10DE02F
:1030700041E0D5E902136A68206802F0BFFC2068CD
:10308000866846F077062068866034E0D5E902134A
:103090006A68206802F0B2FC2068806840F48040D2
:1030A0002168886027E0EA686968206802F0BAFC55
:1030B0005021206802F0ADFC1DE0EA6869682068D4
:1030C00002F0C3FC6021206802F0A3FC13E0EA6870
:1030D0006968206802F0A6FC4021206802F099FC93
:1030E00009E000BF00BF00BF2968206802F091FC22
:1030F00001E0012700BF00BF012084F83D0000BFB0
:10310000002084F83C0000BF384684E7704710B5C3
:10311000044620680069C0F34000D8B12068C06848
:10312000C0F34000B0B16FF00200216808610120D7
:1031300020772068806900F0030018B12046FFF76F
:10314000E5FF05E0204600F0ADF8204600F0ABF8C2
:103150000020207720680069C0F38000D8B1206883
:10316000C068C0F38000B0B16FF00400216808614E
:10317000022020772068806900F4407018B1204652
:10318000FFF7C4FF05E0204600F08CF8204600F071
:103190008AF80020207720680069C0F3C000D8B109
:1031A0002068C068C0F3C000B0B16FF008002168AB
:1031B0000861042020772068C06900F0030018B17E
:1031C0002046FFF7A3FF05E0204600F06BF82046FD
:1031D00000F069F80020207720680069C0F3001033
:1031E000D8B12068C068C0F30010B0B16FF0100013
:1031F00021680861082020772068C06900F44070C9
:1032000018B12046FFF782FF05E0204600F04AF89B
:10321000204600F048F8002020772068006900F080
:10322000010058B12068C06800F0010030B16FF0B3
:10323000010021680861204600F036F82068006926
:10324000C0F3C01058B12068C068C0F3C01030B1DE
:103250006FF08000216808612046FFF7E5FD2068D7
:103260000069C0F3801058B12068C068C0F38010B6
:1032700030B16FF0400021680861204600F020F86E
:1032800020680069C0F3401058B12068C068C0F3DE
:10329000401030B16FF02000216808612046FFF730
:1032A000C4FD10BD7047704710B50446034920683F
:1032B000884201D1FEF7EEFF10BD0000000400407F
:1032C0007047704710B5044600BF00BF21680C313D
:1032D00051E8001F21F4907021680C3141E8000290
:1032E000002AF3D100BF00BF00BF2168143151E8AC
:1032F000001F21F001002168143141E80002002A7A
:10330000F3D100BF206B01280ED100BF00BF2168A0
:103310000C3151E8001F21F0100021680C3141E808
:103320000002002AF3D100BF2068406900F040008D
:1033300000B300BF00BF2168143151E8001F21F025
:1033400040002168143141E80002002AF3D100BF97
:10335000E06B78B10020E16B4863E06BFEF792F917
:1033600040B1E06BFEF78EFA202803D11020606494
:10337000032010BD0020E085202084F842000020BA
:10338000206300BFF5E770B504460025206840695A
:10339000C0F3C01594F84100212817D1B5B100BF82
:1033A00000BF2168143151E8001F21F0800021681E
:1033B000143141E80002002AF3D100BFA06B10B124
:1033C000A06BFEF75FF9204602F037FC20684069E9
:1033D000C0F3801594F84200222817D1B5B100BF80
:1033E00000BF2168143151E8001F21F0400021681E
:1033F000143141E80002002AF3D100BFE06B10B1A4
:10340000E06BFEF73FF9204602F0D1FB002070BDD3
:10341000704700002DE9F84F0446206805682068D1
:10342000C668206847694FF00009CA4605F00F09D1
:10343000B9F1000F0AD105F0200038B106F02000E4
:1034400020B1204602F00CFCBDE8F88FB9F1000F66
:103450007BD007F0010018B906F49070002874D0F2
:1034600005F0010030B106F4807018B1606C40F0D6
:103470000100606405F0040030B107F0010018B1EC
:10348000606C40F00200606405F0020030B107F0AB
:10349000010018B1606C40F00400606405F00800A1
:1034A00048B106F0200010B907F0010018B1606CB7
:1034B00040F008006064606C002845D005F02000F2
:1034C00028B106F0200010B1204602F0C9FB2068A8
:1034D0004069C0F3801A606C00F0080010B9BAF1BE
:1034E000000F2CD0204602F062FB2068406900F0FB
:1034F000400000B300BF00BF2168143151E8001F35
:1035000021F040002168143141E80002002AF3D183
:1035100000BFE06B50B17748E16B4863E06BFEF7AA
:10352000DDF888B1E06B416B88470DE02046FFF77E
:103530006FFF09E009E02046FFF76AFF04E020463C
:10354000FFF766FF002060647EE7206B012877D1DB
:1035500005F01000002873D006F010000028FAD003
:1035600000BF00200090206800680090206840683C
:10357000009000BF00BF2068406900F040000028B4
:103580005FD0E06B006840681FFA80F8B8F1000F68
:1035900055D0A08D404552DDA4F82E80E06B8069A7
:1035A000202843D000BF00BF21680C3151E8001F24
:1035B00021F4807021680C3141E80002002AF3D127
:1035C00000BF00BF00BF2168143151E8001F21F087
:1035D00001002168143141E80002002AF3D100BF44
:1035E00000BF00BF2168143151E8001F21F04000E6
:1035F0002168143141E80002002AF3D100BF2020E5
:1036000084F842000020206300BF00BF21680C3115
:1036100051E8001F21F0100021680C3141E8000240
:10362000002AF3D100BFE06BFEF72CF802206063A4
:10363000A08DE28D801A81B22046FFF742FE03E79B
:1036400042E0A08DE18D401A1FFA80F8E08DD0B3E2
:10365000B8F1000F37D000BF00BF21680C3151E82E
:10366000001F21F4907021680C3141E80002002A0B
:10367000F3D100BF00BF00BF2168143151E8001F23
:1036800021F001002168143141E80002002AF3D141
:1036900000BF202084F842000020206300BF00BF4C
:1036A00021680C3151E8001F21F0100021680C3115
:1036B00041E80002002AF3D100BF022060634146C6
:1036C0002046FFF7FEFDBFE605F0800030B106F0B2
:1036D000800018B1204602F023FCB5E605F040005A
:1036E00030B106F0400018B1204602F096FAABE681
:1036F00000BFA9E6735A000810B504460CB90120B2
:1037000010BDA06900B100E000BF94F8410028B9E5
:10371000002084F84000204600F02AF8242084F895
:1037200041002068C06820F400502168C86020462D
:1037300002F014FB2068006920F4904021680861C1
:103740002068406920F02A00216848612068C0682C
:1037500040F400502168C86000206064202084F894
:10376000410084F842000020606300BFC8E7000009
:1037700010B586B004460020029003900490059096
:103780006249206888426AD100BF6148806940F47C
:1037900080405F4988610846806900F4804001905C
:1037A00000BF00BF00BF0846806940F00400886188
:1037B0000846806900F00400019000BF00BF481572
:1037C0000290022003900320059002A95148FEF7C1
:1037D000A3FB4FF48060029000200390049002A9A4
:1037E0004C48FEF799FB4C484C4908600020486063
:1037F00000214A4881608021C1600021016141614E
:103800008161C161FEF70EFA08B1FDF7B0F900BFA2
:103810004248E063446200BF3F48143840490860B2
:103820001020486000213E4881608021C160002155
:10383000016141618161C161FEF7F4F908B1FDF7F1
:1038400096F900BF3648A063446200BF00220521FC
:103850002520FEF7D9FD2520FEF7C6FD54E03149AD
:103860002068884250D100BF2948C06940F48020B8
:103870002749C8610846C06900F48020019000BF54
:1038800000BF00BF0846806940F008008861084614
:10389000806900F00800019000BF00BF0815029089
:1038A000022003900320059002A91F48FEF734FB75
:1038B0004FF40060029000200390049002A91A487F
:1038C000FEF72AFB14482838184908600020486091
:1038D0000021164881608021C160002101614161A1
:1038E0008161C161FEF79EF908B1FDF740F900BFA3
:1038F0000E48E063446200BF002205212720FEF746
:1039000083FD2720FEF770FD06B010BD0038014092
:103910000010024000080140580002400848002002
:103920004C48002000480040000C01409048002016
:1039300070B504460D46164694F8420020280BD177
:1039400005B10EB9012070BD002020633246294622
:10395000204602F081FAF6E70220F4E76FF020013A
:1039600002681160891002681160704770472DE984
:10397000F84F04460E46174699464FF0000A94F851
:10398000410020284AD106B117B90120BDE8F88FBF
:1039900000206064212084F84100FEF775FC824617
:1039A000A784E784A068B0F5805F04D1206910B9CE
:1039B0000025B04602E035464FF000081BE05346B4
:1039C000002280212046CDF8009002F0D9FA08B1FB
:1039D0000320DBE745B9B8F80000C0F30800216810
:1039E000486008F1020803E02878216848606D1CEF
:1039F000E08C401EE084E08C0028E0D15346002299
:103A000040212046CDF8009002F0BAFA08B1032018
:103A1000BCE7202084F841000020B7E70220B5E78A
:103A200010B5034693F84100202813D101B10AB91B
:103A3000012010BD19629A84DA8400205864212084
:103A400083F841001868C06840F080001C68E0609E
:103A50000020EEE70220ECE76FF020010268116021
:103A6000891002681160704700BFFEE72DE9FC4134
:103A700006460C46082204F110016846FDF758F886
:103A8000208AC0F3C505382D02D2C5F1380001E007
:103A9000C5F1780007463A460A49204600F014FC72
:103AA00008226946204600F00FFC102221463046CD
:103AB000FDF73EF858220021204600F051FCBDE8F9
:103AC000FC8100007C050020002242610261054962
:103AD0000160054941600349C94381600249C94306
:103AE000C16070470123456789ABCDEF2DE9F043F5
:103AF00091B080468946D8F80040D8F80450D8F8EC
:103B00000860D8F80C704022494601A8FCF7F7FF7E
:103B100005EA060027EA0501084301990844FE4921
:103B200008440444E00140EA54642C4404EA0500DB
:103B300026EA0401084302990844F8490844074466
:103B4000380340EA1757274407EA040025EA07012B
:103B5000084303990844F24908440644700440EAC3
:103B6000D6363E4406EA070024EA060108430499D3
:103B70000844EC4908440544A80540EA9525354425
:103B800005EA060027EA0501084305990844E649C5
:103B900008440444E00140EA54642C4404EA05006B
:103BA00026EA0401084306990844E049084407440A
:103BB000380340EA1757274407EA040025EA0701BB
:103BC000084307990844DA4908440644700440EA67
:103BD000D6363E4406EA070024EA0601084308995F
:103BE0000844D44908440544A80540EA95253544CD
:103BF00005EA060027EA0501084309990844CE4969
:103C000008440444E00140EA54642C4404EA0500FA
:103C100026EA040108430A990844C84908440744AD
:103C2000380340EA1757274407EA040025EA07014A
:103C300008430B990844A0F524404F38064470040B
:103C400040EAD6363E4406EA070024EA0601084365
:103C50000C990844BA4908440544A80540EA95254A
:103C6000354405EA060027EA050108430D99084492
:103C7000B44908440444E00140EA54642C4404EA92
:103C8000050026EA040108430E990844AE49084499
:103C90000744380340EA1757274407EA040025EA97
:103CA000070108430F990844A849084406447004D2
:103CB00040EAD6363E4406EA070024EA06010843F5
:103CC00010990844A24908440544A80540EA9525EE
:103CD000354405EA070026EA07010843029908442B
:103CE0009C4908440444600140EAD4642C4404EA3A
:103CF000060025EA06010843079908449649084446
:103D00000744780240EAD757274407EA050024EA27
:103D1000050108430C990844904908440644B0033F
:103D200040EA96463E4406EA040027EA04010843B6
:103D3000019908448A4908440544280540EA153594
:103D4000354405EA070026EA0701084306990844B6
:103D5000844908440444600140EAD4642C4404EAE1
:103D6000060025EA060108430B9908447E490844E9
:103D70000744780240EAD757274407EA050024EAB7
:103D80000501084310990844784908440644B003E3
:103D900040EA96463E4406EA040027EA0401084346
:103DA00005990844724908440544280540EA153538
:103DB000354405EA070026EA070108430A99084442
:103DC0006C4908440444600140EAD4642C4404EA89
:103DD000060025EA060108430F990844664908448D
:103DE0000744780240EAD757274407EA050024EA47
:103DF0000501084304990844604908440644B00397
:103E000040EA96463E4406EA040027EA04010843D5
:103E1000099908445A4908440544280540EA1535DB
:103E2000354405EA070026EA070108430E990844CD
:103E3000544908440444600140EAD4642C4404EA30
:103E4000060025EA06010843039908444E49084440
:103E50000744780240EAD757274407EA050024EAD6
:103E60000501084308990844484908440644B0033A
:103E700040EA96463E4406EA040027EA0401084365
:103E80000D990844424908440544280540EA15357F
:103E9000354485EA06007840069908443D490844BF
:103EA0000444200140EA14742C4484EA0500704064
:103EB00009990844384908440744F80240EA57572A
:103EC000274487EA040068400C99084433490844B1
:103ED0000644300440EA16463E4486EA0700604045
:103EE0000F9908442E4908440544E80540EA552541
:103EF000354485EA06007840029908442949084477
:103F00000444200140EA14742C4484EA0500704003
:103F100005990844244949E078A46AD756B7C7E808
:103F2000DB702024EECEBDC1AF0F7CF52AC68747DB
:103F3000134630A8019546FDD8988069AFF7448BA9
:103F4000BED75C892211906B937198FD8E4379A640
:103F50002108B44962251EF640B340C0515A5E267E
:103F6000AAC7B6E95D102FD65314440281E6A1D842
:103F7000C8FBD3E7E6CDE121D60737C3870DD5F4DB
:103F8000ED145A4505E9E3A9F8A3EFFCD9026F67E0
:103F90008A4C2A8D4239FAFF81F6718722619D6D24
:103FA0000C38E5FD44EABEA4A9CFDE4B0844074423
:103FB000F80240EA5757274487EA04006840089906
:103FC0000844A74908440644300440EA16463E44E3
:103FD00086EA070060400B990844A249084405445A
:103FE000E80540EA5525354485EA060078400E99F3
:103FF00008449D4908440444200140EA14742C44B8
:1040000084EA05007040019908449849084407442F
:10401000F80240EA5757274487EA040068400499A9
:104020000844934908440644300440EA16463E4496
:1040300086EA07006040079908448E490844054411
:10404000E80540EA5525354485EA060078400A9996
:104050000844894908440444200140EA14742C446B
:1040600084EA050070400D990844844908440744D7
:10407000F80240EA5757274487EA0400684010993D
:1040800008447F4908440644300440EA16463E444A
:1040900086EA07006040039908447A4908440544C9
:1040A000E80540EA5525354465EA07007040019966
:1040B0000844754908440444A00140EA94642C442F
:1040C00064EA0600684008990844704908440744B7
:1040D000B80240EA9757274467EA050060400F9905
:1040E00008446B4908440644F00340EA56463E44FF
:1040F00066EA040078400699084466490844054485
:10410000680540EAD525354465EA070070400D99F9
:104110000844614908440444A00140EA94642C44E2
:1041200064EA06006840049908445C49084407446E
:10413000B80240EA9757274467EA050060400B99A8
:104140000844574908440644F00340EA56463E44B2
:1041500066EA04007840029908445249084405443C
:10416000680540EAD525354465EA0700704009999D
:1041700008444D4908440444A00140EA94642C4496
:1041800064EA060068401099084448490844074416
:10419000B80240EA9757274467EA0500604007994C
:1041A0000844434908440644F00340EA56463E4466
:1041B00066EA040078400E9908443E4908440544E4
:1041C000680540EAD525354465EA07007040059941
:1041D0000844394908440444A00140EA94642C444A
:1041E00064EA060068400C990844344908440744CE
:1041F000B80240EA9757274467EA050060400399F0
:1042000008442F4908440644F00340EA56463E4419
:1042100066EA040078400A9908442A49084405449B
:10422000680540EAD5253544D8F800002044C8F890
:104230000000D8F804002844C8F80400D8F80800A2
:104240003044C8F80800D8F80C003844C8F80C000E
:104250004022002101A800F083F811B0BDE8F083EE
:10426000604BBBF670BCBFBEC67E9B28FA27A1EA96
:104270008530EFD4051D880439D0D4D9E599DBE623
:10428000F87CA21F6556ACC4442229F497FF2A4348
:10429000A72394AB39A093FCC3595B6592CC0C8FD8
:1042A0007DF4EFFFD15D84854F7EA86FE0E62CFEA4
:1042B000144301A3A111084E827E53F735F23ABD93
:1042C000BBD2D72A91D386EB2DE9F0470446884626
:1042D0001546208AC0F3C509206900EBC50020619E
:1042E000B0EBC50F02D26069401C6061606900EBF1
:1042F00055716161C9F14007BD421BD304F118013A
:1043000001EB09003A46414600F020F804F118019B
:104310002046FFF7EBFB3E4605E008EB0601204692
:10432000FFF7E4FB403606F13F00A842F5D34FF01B
:10433000000900E00026AA1B08EB060104F118039F
:1043400003EB090000F002F8BDE8F08710B5034662
:10435000002002E00C5C1C54401C9042FAD310BDBB
:1043600010B50346002001E01954401C9042FBD3D5
:1043700010BD00000EB500200090019002901E4874
:104380001E49086081151D488160002101730121CB
:10439000017581614FF46021C161002017494860B7
:1043A000032116480161FCF703FF08B1FCF7DFFBAE
:1043B0000A200090012001900720029069460F48D2
:1043C000FCF7B8FD08B1FCF7D2FB0B2000900220EF
:1043D000019069460948FCF7ADFD08B1FCF7C7FB41
:1043E0000C2000900320019069460448FCF7A2FDD0
:1043F00008B1FCF7BCFB0EBD00240140800F00207B
:1044000008B500BF1248406940F0010010494861FA
:104410000846406900F00100009000BF00BF002284
:1044200005210D20FDF7F0FF0D20FDF7DDFF002237
:1044300005210E20FDF7E8FF0E20FDF7D5FF002235
:1044400005210F20FDF7E0FF0F20FDF7CDFF08BD90
:104450000010024000B59DB01C22184916A8FBF7B9
:10446000E1FE002116A802F0FAFB154908601C22A3
:1044700012491C310FA8FBF7D5FE00210FA802F04E
:10448000EEFB104908601C220C49383108A8FBF7E4
:10449000C9FE002108A802F0E2FB0B4908601C22BB
:1044A0000649543101A8FBF7BDFE002101A802F026
:1044B000D6FB064908601DB000BD0000F080000872
:1044C0008000002084000020880000208C00002054
:1044D00000B585B00020019002900390049000BFC9
:1044E0003A48806940F01000384988610846806980
:1044F00000F01000009000BF00BF00BF08468069B8
:1045000040F0200088610846806900F0200000909B
:1045100000BF00BF00BF0846806940F0040088610A
:104520000846806900F00400009000BF00BF00BF93
:104530000846806940F0080088610846806900F0FC
:104540000800009000BF00BF002241F2790120481E
:10455000FDF794FE4FF6F87001900320029001A938
:104560001C48FDF7D9FCFF20019000200290039029
:1045700001A91948FDF7D0FC41F279000190012012
:104580000290002003900220049001A91048FDF73A
:10459000C3FC4EF2863001900320029001A90C4822
:1045A000FDF7BAFC4FF4194001900320029001A9D5
:1045B0000948FDF7B1FC042001900320029001A9F5
:1045C0000648FDF7A9FC05B000BD00000010024040
:1045D000000C01400010014000080140001401409F
:1045E00000B587B0002003900490059006900190DC
:1045F00002904FF080401549086040F21F3048603B
:1046000000211248816041F63F71C16000210161C3
:1046100080218161FEF758FC08B1FCF7A8FA4FF43D
:104620008050039003A90948FEF7EAFC08B1FCF7A3
:104630009EFA00200190029001A90448FEF7F6FBC3
:1046400008B1FCF794FA07B000BD000084320020E6
:1046500010B50B480B4908604FF416504860002114
:1046600008488160C16001610C21416100218161C4
:10467000C161FFF741F808B1FCF779FA10BD0000FD
:10468000003801407847002010B50B480B490860FE
:104690004FF416504860002108488160C1600161F4
:1046A0000C21416100218161C161FFF725F808B14A
:1046B000FCF75DFA10BD000000480040C047002034
:1046C00000BFFEE710B586B0FE480078012831D162
:1046D0000621FD4801F082FFFB498979FA4AD27927
:1046E00041EA02218842F2D1F84800880A2821DAFA
:1046F000F5480078F649097888421CD1F24840789C
:10470000032818D1F0488078A8B9EF48C07801286C
:1047100011D1ED48007970B9EB48407901280AD1F0
:1047200007200090EB48037802220321E848008824
:1047300002F0E6FE11E2E4480078E5490978884293
:104740001CD1E1484078032818D1DF488078A8B907
:10475000DD48C078022811D1DB48007970B9DA4809
:10476000407901280AD107200090DB480378022213
:104770000321D748008802F0C3FEE1E3D248007865
:10478000D349097888421CD1CF484078032818D1F2
:10479000CD488078A8B9CC48C078032811D1CA4840
:1047A000007970B9C848407901280AD107200090E3
:1047B000CA48038802220321C548008802F0A0FEEF
:1047C000BEE3C1480078C249097888421CD1BE487E
:1047D0004078032818D1BC488078A8B9BA48C07876
:1047E000042811D1B848007970B9B7484079012838
:1047F0000AD107200090BA48038802220321B44856
:10480000008802F07DFE9BE3AF480078B04909784C
:1048100088421CD1AC484078032818D1AA48807837
:10482000A8B9A948C078052811D1A748007970B95E
:10483000A548407901280AD107200090A94803889B
:1048400002220321A248008802F05AFE78E39E4823
:1048500000789F49097888421FD19B4840780328F7
:104860001BD199488078C0B99748C078012814D1E5
:104870009548007988B99448407902280DD10920DB
:1048800095490978CDE90010924803780422032164
:104890008F48008802F09EFE52E38B4800788C49D6
:1048A0000978884222D18848407803281ED186485A
:1048B0008078D8B98448C078012817D18248007917
:1048C000A0B981484079032810D10B218348008882
:1048D000814A1278CDE9002002917E4803780622B1
:1048E00003217B48008802F013FD29E37648007815
:1048F00077490978884225D173484078032821D127
:1049000071488078F0B97048C07801281AD16E4893
:104910000079B8B96C484079042813D10D2070494A
:104920000A886E4909886C4B1B78CDE90031CDE9C6
:10493000022068480378082203216548008802F0B5
:104940002FFDFDE26048007861490978884228D14E
:104950005D484078032824D15B48807808BB5A48DA
:10496000C07801281DD158480079D0B956484079FF
:10497000052816D10F225B48018859480088574BFB
:104980001B88CDE90130CDE903125348007800902F
:10499000504803780A2203214D48008802F054FD54
:1049A000CEE2494800784A49097888421FD14648F2
:1049B000407803281BD144488078C0B94248C07869
:1049C000022814D14048007988B93F48407902282C
:1049D0000DD1092041490988CDE900103E480378EE
:1049E000042203213A48008802F0F4FDA8E2364888
:1049F000007837490978884222D133484078032823
:104A00001ED131488078D8B92F48C078022817D1F4
:104A10002D480079A0B92C484079032810D10B21EA
:104A20002F4800882D4A1288CDE9002002912A489B
:104A30000378062203212648008802F069FC7FE201
:104A40002148007822490978884225D11E484078BB
:104A5000032821D11C488078F0B91B48C07802286F
:104A60001AD119480079B8B917484079042813D1E8
:104A70000D221C4800881A490988184B1B88CDE96B
:104A80000031CDE9020214480378082203211048BE
:104A9000008802F085FC53E20B4800780C49097845
:104AA000884232D10848407803282ED106488078C1
:104AB00058BB0548C078032827D10348007920BB9C
:104AC000014811E041050020CC3A002042050020B9
:104AD000720000207C0000207D0000209600002055
:104AE0009800002094000020407902280DD1092070
:104AF000FE490988CDE90010FD48038804220321FE
:104B0000FC48008802F066FD1AE2FB480078F9498B
:104B10000978884222D1F848407803281ED1F64807
:104B20008078D8B9F448C078032817D1F2480079C2
:104B3000A0B9F1484079032810D10B20EF4909882A
:104B4000EA4A1288CDE900210290E948038806224A
:104B50000321E848008802F0DBFBF1E1E648007839
:104B6000E449097888421FD1E348407803281BD1E3
:104B7000E1488078C0B9E048C078042814D1DE4804
:104B8000007988B9DC48407902280DD10920DB4939
:104B90000988CDE90010D548038804220321D548AF
:104BA000008802F017FDCBE1D3480078FA281BD12A
:104BB000D1484078032817D1CF488078A0B9CE4893
:104BC000C078AA2810D1CC48007968B9CA48407981
:104BD000012809D107200090C6480388022203213A
:104BE000FA2002F08DFCABE1C3480078C149097896
:104BF000884224D1C0484078032820D1BE4880781C
:104C000050281CD1BC48C078C8B9BB480079B0B99D
:104C1000B9484079022812D10921B948008880B2E8
:104C2000CDE90001B64800684FF6FF7101EA104374
:104C300004220321AF48008802F0CCFC80E1AE489A
:104C40000078AC490978884228D1AB4840780328DD
:104C500024D1A9488078502820D1A748C0780228BC
:104C60001CD1A5480079C8B9A3484079022815D1BC
:104C7000A44802F0D9FD0921A348008880B2CDE9FB
:104C80000001A14800684FF6FF7101EA10430422B9
:104C900003219848008802F09DFC51E19648007875
:104CA00094490978884220D19348407803281CD140
:104CB00091488078502818D18F48C078042814D1A2
:104CC0008D48007988B98C48407901280DD18D48EC
:104CD00002F0BEFD072000908C48038802220321C9
:104CE0008448008802F00CFC2AE18348007881495E
:104CF0000978884229D180484078062825D17E4805
:104D0000807810BB7C48C07802281ED17A48007990
:104D1000D8B97949487902F0D7FC052276497C4810
:104D200001F0CCF974484079734C247940EA0423AB
:104D30007148C078704CA47840EA04226E484178EB
:104D40006C48008802F012FCFAE06B480078694970
:104D50000978884229D168484078062825D16648D4
:104D6000807810BB6448C0780A281ED16248007958
:104D7000D8B961484079012817D100225E496548B9
:104D800001F09CF95C4840795B4C247940EA0423AB
:104D90005948C078584CA47840EA042256484178D3
:104DA0005448008802F0E2FBCAE0534800785149B9
:104DB0000978884229D150484078062825D14E48A4
:104DC000807810BB4C48C0780B281ED14A48007927
:104DD000D8B949484079012817D1002246494E48A0
:104DE00001F06CF944484079434C247940EA0423AB
:104DF0004148C078404CA47840EA04223E484178BB
:104E00003C48008802F0B2FB9AE03B480078394900
:104E10000978884229D138484078062825D1364873
:104E2000807810BB3448C0780C281ED132480079F5
:104E3000D8B93149487902F07DFC05222E4937481E
:104E400001F03CF92C4840792B4C247940EA0423AA
:104E50002948C078284CA47840EA042226484178A2
:104E60002448008802F082FB6AE023480078214948
:104E70000978884225D120484078062821D11E484B
:104E80008078F0B91C48C078AA281AD11A4800794D
:104E9000B8B905221849224801F010F9164840799E
:104EA000154C247940EA04231348C078124CA478A6
:104EB00040EA0422104841780E48008802F056FB70
:104EC0003EE00D4800780B490978884234D10A4801
:104ED0004078062830D10848807868BB0648C078FA
:104EE000CC2829D104480079A5281BE0980000208F
:104EF0009600002072000020CC3A00209400002090
:104F000078000020003007083C000020400000200E
:104F10000008070800180708002007080010070805
:104F20000000070808D1074840795A2804D101F049
:104F30008DFBFDF7BBFA03E001F088FB02F0AAF954
:104F400006B010BDCC3A002000BFFEE7FEB5002041
:104F5000FE490870FE48407AFD49097A40EA01207E
:104F6000FC490880FA48C078F949897840EA01206C
:104F7000F9490880F9480588F9A103C9CDE901017B
:104F8000F348C079F84908704FF48061F748FBF79F
:104F900062F94FF48061F648FBF75DF9F54802F0DD
:104FA00043FCF1480078012804D002287ED0042870
:104FB0007DD126E22822E6490A31EF48FBF732F993
:104FC0008021E3480A3001F079FBEC490880E81EB3
:104FD000DF49095C281FDE4A105C41EA0020E849ED
:104FE00008800020E7490860E4480088E44909880F
:104FF00088427DD100240AE0E3482044017904F18D
:105000000A00D34A105C814200D002E0641C582C94
:10501000F2DB00BF322C6CDA00240FE00A2000EB38
:105020004400CB49085C0B2101EB4401C84A515CA8
:1050300040EA0120CD4921F81400641C192CEDDB55
:105040001922D149091DC948FBF75CFE322001F045
:1050500056FB0120CD490860CB491B31CC4802F0FA
:1050600029F9CA48006868B3C948007800F00F0001
:1050700042F210714843C649497801F00F0101EB33
:105080004102C2EBC11100EBC100C149897801F0B6
:105090000F0101EBC10202EB011100EB8100BC49E1
:1050A000C97801F00F0101EB810101E0BCE021E2D0
:1050B00000EB4100B649097901F00F010844B549F8
:1050C000086022E0B248007800F00F004FF47A71D7
:1050D0004843AF49497801F00F0101EBC10202EBEF
:1050E000011100EB8100AA49897801F00F0101E06C
:1050F00080E061E001EB810100EB4101A448C07850
:1051000000F00F000844A3490860A2480068A249C3
:105110000860A24801F0FCFAFCF7E6FE9E48002376
:105120009E4902680120FCF787FEFCF77BFE97484A
:105130000068F8B11022944921319948FBF7CCFD61
:10514000082298499648FBF7DDFD00200FE09449BE
:1051500031F810104FF47F4202EA0121904A32F8F0
:10516000102041EA12218E4A22F81010401C082813
:10517000EDDB1EE01022844920318948FBF7ACFDAD
:10518000082288498648FBF7BDFD00200FE08449CE
:1051900031F810104FF47F4202EA0121804A32F8C0
:1051A000102041EA12217E4A22F81010401C0828E3
:1051B000EDDB7D48734908604FF480616448FBF77C
:1051C0004AF8502001F09BFA78488079009077489F
:1051D0004079764E367940EA06237448C078734E9B
:1051E000B67840EA0622714841787148008802F09A
:1051F00031FA0EE04FF480615548FBF72CF801A816
:10520000FBF734F886B26423324601A96948FEF7F9
:10521000AEFB4FF480615548FBF71DF84FF48061F9
:105220005348FBF718F866E1802149480A3001F03D
:1052300045FA52490880E81E4549095C281F444A3E
:10524000105C01EB00204E4908805B480068401C60
:1052500018B955484B4908600BE0574E3068524921
:105260008022461A96FBF2F3464E3060394F3B805F
:1052700000BF4248008842490988884259D1002429
:105280000FE00A2000EB44003149085C0B2101EBE0
:1052900044012F4A515C40EA0120344921F81400AE
:1052A000641C402CEDDB4022364801682F48FBF798
:1052B00029FD3448006880303249086001221146D7
:1052C0003E48FCF7DBFF0120FCF740FD00220121F6
:1052D0003A48FCF7D3FF1E48C0781D49897840EA58
:1052E00001202849098889B288420AD001A8FAF722
:1052F000BDFF86B26423324601A92E48FEF737FB74
:10530000F9E04FF480611248FAF7A5FF1D480068E4
:105310002B490860084600684FF6FF7101EA10400B
:10532000284908802648008848800A480088401C90
:105330008880012211462148FCF7A0FF0120FCF7DC
:1053400005FD002201211D483EE00000400500202F
:10535000CC3200201600002018000020420500205A
:105360006572726F720D0A0004000020B6060020FC
:10537000B60A002000300708340600201E00002076
:1053800020000020240000207AF0070834000020CC
:105390007C06002028000020540000200048070858
:1053A000960600200050070800000408CC3A0020B0
:1053B00072000020784700203C000020000C0140D3
:1053C0003800002048000020FCF758FF03224B491A
:1053D0004B48FBF797FC4B4880790090494840794F
:1053E000484E367940EA06234648C078454EB6789E
:1053F00040EA0622434841784348008802F02AF9EF
:1054000079E08021414801F059F941490880E81EBE
:105410003E490A39095C281F3C4A0A3A105C01EBF4
:1054200000203C4908803A4800880988884250D1C9
:10543000082239493948FBF74FFC00200FE0374973
:1054400031F810104FF47F4202EA0121334A32F85A
:10545000102041EA1221314A22F81010401C042881
:10546000EDDB2F492D4801F00BF92E4801F050F9E2
:10547000FCF73AFD2A4800232A4902680220FCF77B
:10548000DBFCFCF7CFFC284801682848FBF760FAF2
:10549000274908600846006810B100F08FF828E03E
:1054A00024A11A480A3800F0B3FE0646502001F045
:1054B00026F9B2B215490A392248FEF7B1FA02E0DC
:1054C0000120FCF743FC1F4890F841002128F7D049
:1054D0000FE0502001F013F901A8FAF7C7FE86B2D9
:1054E0006423324601A91748FEF741FA502001F023
:1054F00006F900E000BF00BFFEBD00000030070855
:1055000048000020CC3A002072000020D632002053
:105510001E0000202000002088F007080600002060
:105520007800002000400708540000200000040814
:1055300030000020636865636B3D6572726F720DA9
:105540000A0000007847002008B508490968C90822
:105550004FF47A72B1FBF2F14143009100BF00BFFA
:1055600000994A1E00920029F9D108BDC805002003
:1055700070B504460D4629462046FCF76DFE08B975
:10558000012070BD0020FCE708B509480949086002
:105590000846008880B2ADF8020008460068000C9A
:1055A000ADF80000022204496846FBF7ABFB08BDDA
:1055B000BBBB55552C0000207AF0070808B54FF00A
:1055C000AA30194908600846008880B2ADF800008A
:1055D0000846008880B2ADF80200084600680090D6
:1055E000042212496846FBF78DFB00BF00BF00BFD5
:1055F00000BF00BFBFF34F8F00BF00BF00BF0C480C
:10560000006800F4E0600B490843001D0849086089
:1056100000BF00BF00BFBFF34F8F00BF00BF00BF80
:1056200000BF00BFFDE700002C0000207AF0070853
:105630000CED00E00000FA0500BF012001F0FEFAC9
:10564000012211460B48FCF719FE0120FCF77EFBF6
:10565000002201210748FCF711FEFBF735FC064943
:105660000870FBF75DFC054908700548FBF78EFBE9
:10567000E3E70000000C01407C0000207D000020DA
:10568000800F002000BF012001F0D8FAFBE700BF27
:10569000012001F0D3FAFBE738B502224C496846F5
:1056A000FBF71AFBBDF80200BDF8001040EA01400C
:1056B0004849086048480068484908604FF48061DC
:1056C0004748FAF7C8FD474802F04AF841480068E1
:1056D000B0F1AA3F08D0B0F1BB3F04D04249084422
:1056E000002870D15BE06FE03B4800683B490860F0
:1056F000084601683D48FBF72BF90546E5B13748F8
:105700003A4902683A4801F069F95020FCF71EFB5B
:1057100038A1334800F07CFD0446A2B23049384835
:10572000FEF77EF902E00120FCF710FB344890F808
:1057300041002128F7D016E032A1294800F068FD89
:105740000446502000F0DBFFA2B225492C48FEF7AA
:1057500067F902E00120FCF7F9FA294890F84100C6
:105760002128F7D038BD1D4801682148FBF7F0F823
:10577000A0B127A11A4800F04BFD0446A2B2184977
:105780001F48FEF74DF902E00120FCF7DFFA1C4844
:1057900090F841002128F7D0FFF7F6FE00BF0F4830
:1057A0000068B0F5003F0CD20C4801681048FBF7C8
:1057B000CFF830B1002080F3138800BF0C4801F00F
:1057C00091F901E0FFE7CDE700BF00BFCAE70000A5
:1057D0007AF007085C000020280000205400002018
:1057E000CC320020004807084544AAAA000004085B
:1057F000000002087570646174696E670000000043
:1058000078470020636865636B6661696C0000001F
:10581000636865636B6F6B0000BF012001F00EFAD7
:105820001248007801281ED1114800888E281AD10C
:105830001048007810490978884214D10D48407802
:10584000102810D18C210D4800F0C8FE094991F8AC
:105850008C10084A92F88D2041EA0221884202D138
:10586000FFF774FBD9E7FEF72DFFD6E740050020D0
:1058700042050020CC3A002072000020CC320020EB
:1058800010B500BF502080F31188BFF34F8FBFF3D6
:105890006F8F00BF02F0E6FA18B14FF08050044954
:1058A000086000BF002080F3118800BF10BD000019
:1058B00004ED00E000B595B028210BA8FAF7CBFC69
:1058C000142106A8FAF7C7FC18216846FAF7C3FCAA
:1058D00001200B9000040C9000200D9001200F90EF
:1058E00002201290C1031391002114910BA8FDF71F
:1058F00069F808B1FBF73BF90F20069002200790EA
:1059000080200890C000099000200A90002106A87D
:10591000FCF712FF08B1FBF72AF9022000904003C0
:1059200002906846FCF770FE08B1FBF720F915B04D
:1059300000BD704710B54FF480510348FCF794FC4C
:105940000248FDF7E4FB10BD000C0140843200204A
:1059500010B50248FDF7DBFB10BD0000D448002065
:1059600010B50268204B98420ED0204B98420BD0C5
:10597000B0F1804F08D01E4B984205D01D4B984285
:1059800002D01D4B984203D122F070024B681A439B
:10599000154B98420ED0154B98420BD0B0F1804F6A
:1059A00008D0134B984205D0124B984202D0124BAC
:1059B000984203D122F44072CB681A4322F080034C
:1059C0004C6943EA040202608B68C3620B6883621D
:1059D000054B984202D0054B984201D10B690363F5
:1059E0000123436110BD0000002C01400034014040
:1059F0000004004000080040000C004030B50C4698
:105A0000816821F47F4142EA0325254329438160CF
:105A100030BD0A46816821F0700142F00703194346
:105A20008160704730B50B461446026A056A25F05E
:105A300001050562816921F0F00141EA041122F0BB
:105A40000A021A438161026230BD30B50B4614462A
:105A5000026A056A25F010050562816921F470412A
:105A600041EA043122F0A00242EA0312816102629B
:105A700030BD70B505466C6A0020E085E0842046A4
:105A8000FDF7C6FC70BD70B506460025746A206837
:105A90004069C0F3C01594F84100212805D125B113
:105AA0000020E084204600F0C8F820684069C0F378
:105AB000801594F84200222805D125B10020E08508
:105AC000204600F074F8606C40F0100060642046DE
:105AD000FDF79EFC70BD70B505466C6A28680068CD
:105AE00000F02000002842D1E08500BF00BF2168FF
:105AF0000C3151E8001F21F4807021680C3141E81D
:105B00000002002AF3D100BF00BF00BF216814319A
:105B100051E8001F21F001002168143141E8000222
:105B2000002AF3D100BF00BF00BF2168143151E843
:105B3000001F21F040002168143141E80002002AD2
:105B4000F3D100BF202084F84200206B01280ED141
:105B500000BF00BF21680C3151E8001F21F0100088
:105B600021680C3141E80002002AF3D100BF002077
:105B70006063206B012804D1A18D2046FDF7A1FBB5
:105B800002E02046FDF7EAFE70BD70B505466C6A7E
:105B900001206063206B012805D1A08D41082046BB
:105BA000FDF78FFB02E02046FDF7E0FE70BD00BF71
:105BB00000BF02680C3252E8002F22F49071026894
:105BC0000C3242E80013002BF3D100BF00BF00BF2E
:105BD0000268143252E8002F22F0010102681432E8
:105BE00042E80013002BF3D100BF016B01290ED155
:105BF00000BF00BF02680C3252E8002F22F01001F3
:105C000002680C3242E80013002BF3D100BF2021C0
:105C100080F8421000210163704710B504462068E7
:105C2000C06820F040002168C860202084F841004E
:105C30002046FDF711FF002010BD00BF00BF026825
:105C40000C3252E8002F22F0C00102680C3242E808
:105C50000013002BF3D100BF202180F841107047C2
:105C6000F8B5044694F84200222875D1A068B0F532
:105C7000805F0CD1206950B90025A66A2068406871
:105C8000C0F308003080A06A801CA06215E0A56AFD
:105C90000026A068B0F5805F03D0A06828B920690D
:105CA00018B920684068287004E02068406800F057
:105CB0007F002870A06A401CA062E08D401E80B268
:105CC000E085002846D12068C06820F020002168C7
:105CD000C8602068C06820F480702168C8602068AF
:105CE000406920F0010021684861202084F84200CA
:105CF00000206063206B012826D10020206300BFB4
:105D000000BF21680C3151E8001F21F0100021680C
:105D10000C3141E80002002AF3D100BF206800687E
:105D200000F0100010280AD100BF00200090206869
:105D30000068009020684068009000BF00BFA18DFF
:105D40002046FDF7BEFA02E02046FDF707FE0020E0
:105D5000F8BD01E00020FBE70220F9E770B504463A
:105D60002168096921F44051E268114322681161F8
:105D70002269A1681143626941EA02052168C96884
:105D800041F20C62914329432268D160216849693C
:105D900021F44071A2691143226851612D4A2168A2
:105DA000914202D1FCF7C6FD01E0FCF7B3FD00EB28
:105DB000C00101EB001162689200B1FBF2F100EB4F
:105DC000C00202EB001263689B00B2FBF3F2642393
:105DD000B2FBF3F202EBC20303EB0212A1EB82016E
:105DE000322202EB01116422B1FBF2F101F0F00169
:105DF00000EBC00202EB001263689B00B2FBF3F2FF
:105E00006423B2FBF3F201EB021200EBC00101EBE1
:105E1000001163689B00B1FBF3F100EBC00303EBDF
:105E200000136668B600B3FBF6F36426B3FBF6F323
:105E300003EBC30606EB0313A1EB8301322303EB51
:105E400001116423B1FBF3F101F00F011144226849
:105E5000916070BD0038014077B581B004461546A9
:105E60000298A062A58500206064222084F8420088
:105E70002848E16B88622848E16BC8622748E16BDB
:105E800008630020E16B486302AE32682368191D85
:105E90002B46E06BFBF70CFF00BF00200090206852
:105EA0000068009020684068009000BF00BF206933
:105EB00070B100BF00BF21680C3151E8001F41F4F0
:105EC000807021680C3141E80002002AF3D100BF44
:105ED00000BF00BF2168143151E8001F41F00100EC
:105EE0002168143141E80002002AF3D100BF00BF4D
:105EF00000BF2168143151E8001F41F040002168C3
:105F0000143141E80002002AF3D100BF002004B0A0
:105F100070BD0000D75A00088B5B0008875A000844
:105F2000014691F84100212828D18868B0F5805FAA
:105F30000BD1086948B90A6A1088C0F308000B68D9
:105F40005860086A801C086205E00B6A581C0862E9
:105F500018780B685860C88C401E80B2C88458B945
:105F60000868C06820F080000B68D8600868C068C6
:105F700040F040000B68D860002070470220FCE72A
:105F80002DE9F04104460D4617469846069E34E03A
:105F9000701C88B32EB1FCF777F9A0EB0800B04273
:105FA0002BD900BF00BF21680C3151E8001F21F43C
:105FB000D07021680C3141E80002002AF3D100BF03
:105FC00000BF00BF2168143151E8001F21F001001B
:105FD0002168143141E80002002AF3D100BF2020DB
:105FE00084F8410084F8420000BF002084F840009B
:105FF00000BF0320BDE8F081FFE72068006828406B
:10600000A84201D1012000E00020B842C0D0002009
:10601000F0E7000008B51C4800680068C0F30010F5
:1060200068B300BF00200090174800680068009027
:10603000154800684068009000BF00BF1248FDF797
:10604000A2F9124800684068C0F5806010490880D5
:10605000084602880F491048FAF7E4F80C4802880D
:106060000C490E48FAF7DEF84FF4806209490648F9
:10607000FDF75EFC01200A4908700A4908700248D1
:10608000FDF7C8F908BD0000784700200848002047
:1060900042050020CC360020CC320020CC3A002033
:1060A000400500204105002010B50248FDF7B2F977
:1060B00010BD0000C047002000BFFEE72DE9F047FB
:1060C00005460F4690460024284600F021FBFBF7CA
:1060D0000BFF414885420CD117F8084022460023A7
:1060E00001460120FBF7A8FE06460EB93B48048096
:1060F0006EE03B4885420CD117F808402246002349
:1061000001460120FBF798FE06460EB935490C7092
:106110005EE0354885420CD117F80840224600233E
:1061200001460120FBF788FE06460EB92F48048081
:106130004EE02F48854202D02E48854248D14FF488
:106140003A762B4885421FD12B480088B04204DBA9
:1061500029480088801B84B205E027480088301A4F
:1061600084B244F400442246002321490120FBF775
:1061700063FE8146B9F1000F05D1C4F30E001F493B
:1061800008801F48048022E01A4885421FD11D481C
:106190000088B04204DB1B480088801B84B205E005
:1061A00018480088301A84B244F400442246002380
:1061B00010490120FBF740FE8146B9F1000F05D1DF
:1061C000C4F30E00104908801048048000BF00BFCF
:1061D000FBF728FEBDE8F0870000070872000020EA
:1061E000000807087D000020001007087400002048
:1061F00000180708002007089E000020A2000020C9
:1062000090000020A0000020A400002092000020A8
:106210000FB4084B10B504A902AA039800F038F88F
:10622000044602A9002000F0D4F9204610BC5DF815
:1062300014FB0000D365000802480068C0F3022088
:10624000704700000CED00E010B5002804DB0A07E1
:10625000130E054A135406E00A07140E034A00F011
:106260000F031B1FD45410BD00E400E018ED00E044
:1062700002E008C8121F08C1002AFAD1704770470F
:10628000002001E001C1121F002AFBD1704700006D
:106290002DE9FF4F8BB088460546002606E02528ED
:1062A0000BD0DDE90D1290476D1C761C2878002874
:1062B000F5D10FB03046BDE8F08F0024A146A246CC
:1062C0000122AE4900E0044315F8013F203B02FAE9
:1062D00003F00842F7D128782A2810D06FF02F0257
:1062E0002878A0F13001092915D809EB890102EBC2
:1062F000410144F0020400EB01096D1CF0E758F87D
:10630000041B5FEA010903D544F40054C9F10009F4
:1063100044F002046D1C28782E2817D115F8010FBF
:1063200044F004042A280ED06FF02F022878A0F140
:10633000300109290AD80AEB8A0102EB410100EB7E
:10634000010A6D1CF2E758F804AB6D1C28786C2824
:106350000FD006DC4C2817D068280DD06A2814D13D
:1063600004E0742810D07A280FD10DE044F4001412
:106370000AE044F4801401E044F440146978814256
:1063800002D104F580146D1C6D1C2878692865D035
:1063900006DC00288DD0632827D0642806D15DE074
:1063A0006E2808D073282AD0752877D0DDE90D1221
:1063B0009047761CE0E0C4F30250022809D003287D
:1063C0000DD0D8F8001004280DD00E6008F1040894
:1063D000D2E0D8F80010F217C1E90062F6E7D8F869
:1063E00000100E80F2E70E70F0E718F8041B8DF82D
:1063F000001000208DF80100EB46012003E058F862
:1064000004BB4FF0FF3061074FF0000701D40AE0F2
:106410007F1C57450DDA8742FADB1BF8071000296D
:10642000F6D106E07F1C8742FCDB1BF80710002931
:10643000F8D1DDE90D23A9EB07008146214600F0E4
:10644000B1F83044C61904E0DDE90D121BF8010B68
:1064500090477F1EF8D22146484688E058F8040B42
:10646000C4F302514FF00A0B032900D100B20429F2
:1064700000D140B2002802DA40422D2102E021057D
:1064800005D52B218DF82410012104E006E0E10759
:1064900010D02021F6E708AF089113E058F8040B5C
:1064A000C4F302514FF00A0B032900D180B2042932
:1064B00000D1C0B20021EEE75946FAF797F8303123
:1064C00007F8011D0028F7D1ADEB070000F1200B04
:1064D000600702D524F4803401E04FF0010ADA4568
:1064E00002DDAAEB0B0000E00020824600EB0B016E
:1064F00008980144A9EB01000A90E00306D4DDE905
:106500000D2321460A9800F04DF806444FF000098B
:1065100008E009A911F80900DDE90D12904709F119
:106520000109761C08998945F3DBE0030CD5DDE908
:106530000D2321460A9800F035F8064404E0DDE911
:106540000D1230209047761CBAF10001AAF1010A21
:10655000F5DC05E0DDE90D1217F8010B9047761C1C
:10656000BBF10001ABF1010BF4DC0A982146DDE937
:106570000D2300F005F806446D1C97E6092801007C
:106580002DE9F041044600251E461746880404D430
:1065900005E039462020B0476D1C641EF9D5284619
:1065A000BDE8F0812DE9F041044600251E469046E5
:1065B000C80301D5302700E02027880404D505E072
:1065C00041463846B0476D1C641EF9D52846BDE8E3
:1065D000F0810A68531C0B601070704730B502469A
:1065E0000B464FF6FF70002110E0545C6040002421
:1065F00009E000F0010525B14AF2010585EA6000D5
:1066000000E04010641C082CF3DB491C9942ECDBD1
:1066100030BD000010B504460B480068C06820F487
:10662000005009490968C86007484460FDF764F8EC
:1066300008B1FAF79CFA04480068C06840F40050BA
:1066400001490968C86010BD7847002010B54FF4B3
:1066500080610748F9F7FFFD4FF480610548F9F7BD
:10666000FAFD0020044908700449087010BD0000BC
:10667000CC3A0020CC360020410500204005002007
:1066800010B50288C2F30323027863F31F121306C6
:106690004288C2F3032464F31F1243EA0243828850
:1066A000C2F3032464F31F1243EA0223C288C2F335
:1066B000032464F31F1213430B6010BD30B5024670
:1066C0000B460020002117E0545C80EA04200024DF
:1066D0000EE000F400452DB141F2210585EA4005A8
:1066E000A8B203E04FF6FF7505EA4000651CECB266
:1066F000082CEEDB4C1CA1B29942E5DB30BDC20098
:10670000002100BF01E000BF491C9142FBD370474C
:1067100030B585B004460020019003940120049018
:1067200000200090FBF7E0FB694601A8FBF722FB85
:106730000546FBF777FB15BB1248844203D10020C6
:10674000114908801BE01148844203D10020104900
:10675000087014E00F48844204D14FF6FF700E49D0
:1067600008800CE00D48844203D100200C490880C9
:1067700005E00C48844202D100200B49088005B096
:1067800030BD000000000708720000200008070864
:106790007D00002000100708740000200018070882
:1067A000A200002000200708A40000202DE9FF4FD0
:1067B0008BB08B4690469946199E0020089009F1AF
:1067C000010258F8221058F82900F9F7A8FD82466E
:1067D0006649F9F7DCFD07900A960A9EB00000F0C2
:1067E000F7F904464FF0000A12E05046F9F77FFE31
:1067F00003900799F9F799FD049009F1010058F801
:1068000020100498F9F739FD44F82A000AF1010A2A
:10681000B245EADB4FF0FF35554806904FF0000ACD
:1068200022E054F82A100B98F9F779FD0190F9F756
:1068300099FE21F00041CDE90201F9F7A6FE04908E
:1068400006990498F9F7BEFE01D2504600E02846AA
:10685000054606990498F9F7B5FE01D2049800E0C0
:10686000069806900AF1010AB245DADB4148059024
:106870000996099EB00000F0ABF907464FF0000AF8
:1068800011E05046F9F733FE3A490390F9F74DFD10
:10689000049018985BF820100498F9F7EEFC47F87C
:1068A0002A000AF1010AB245EBDB54F8250032490F
:1068B000F9F792FE04D248F29010304908804AE07D
:1068C00054F825002E49F9F787FE1FD254F8250009
:1068D0002949F9F777FE19D857F82500F9F742FE4C
:1068E00021F000410022274BCDE90001F9F78DFD91
:1068F000CDE90201F9F71DFE80B20890089840F436
:10690000004008901D490898088024E054F82500AC
:106910001D49F9F761FE10D854F825001849F9F718
:1069200051FE0AD857F825001049F9F7FEFC8246B7
:10693000F9F7EBFD114908800DE054F825001249E4
:10694000F9F740FE04D240F21A400C49088002E0F8
:1069500000200A49088000200890384600F016F808
:10696000204600F013F80FB0BDE8F08F0000204182
:1069700000007A44CDCCCC3DB57DAA433C05002037
:10698000E9F70242000024408104153F10B50028B9
:1069900021D0114B0022001F196803E0814203D867
:1069A0000A4649680029F9D152B11368841A9C42F9
:1069B00004D1006818441060104602E0506000E006
:1069C000186039B102680B1A934203D10B681A445C
:1069D00002604968416010BD2C0600202DE9FC478B
:1069E00081460C461546AFB2264632483249086009
:1069F00007F50060C11700EB5151C9122F4A1180F1
:106A00004FF400612E48F9F726FC2EA103C9CDE909
:106A1000000101202D49086044E0012211462C4864
:106A2000FBF72CFC0520FBF791F9002201212848F7
:106A3000FBF724FC4FF4006231462148FAF74CF989
:106A40004FF480621C4801681D48FAF75BF950203A
:106A5000FFF755FE1D486A461EA103681F48FFF751
:106A6000D7FB80461FFA88F21C491D48FCF7D8FF67
:106A700006F500661048006800F500600E490860E1
:106A8000012211461248FBF7F9FB0520FBF75EF9DE
:106A9000002201210E48FBF7F1FB0C480068401C66
:106AA0000A49086009480068044909888842B4DD39
:106AB000BDE8FC87000002086400002060000020A0
:106AC0000020002061636B3D000000006800002092
:106AD000000C01402573256400000000CC3200202A
:106AE0007847002070B5044672B6206880F30888A5
:106AF00000BF6568A84770BDFBF7D8FBFEF7DAFE5C
:106B0000FDF7E6FCFDF77CFCFDF7A2FDFDF732FC8E
:106B1000FDF766FDFDF7B8FD1E48FCF729FA1E4893
:106B200000F01EFEFEF7B8FDF9F7D4FE1B4800F09A
:106B30009FFE1A480E3000F049FE194800F0D4FBC1
:106B4000184800F0CDFB054600F0BEFD164800F0E9
:106B5000C7FB054600F0EEFD14A11648FFF758FBF1
:106B60000446A2B213491448FCF75AFF4FF480625E
:106B700012491148FCF7DCFE0F480068C06840F07D
:106B800010000D490968C860FDF764FC00F062F868
:106B900000BFFEE784320020004807087AF00708AB
:106BA000000007080008070800100708617070312E
:106BB00000000000CC32002078470020CC360020B6
:106BC00001460020842901D0CA1C104470470000EF
:106BD000F0B50B30154D20F007010024144A0FE0EA
:106BE00003688B420BD38B4205D95E1A4318476862
:106BF000C3E9006700E04368136002C004E0021DBF
:106C000010680028ECD12046002802D1286808B17D
:106C10000020F0BD064A07481060074A121A22F009
:106C20000702C0E9002401202860D7E730060020D1
:106C30002C060020345600203058002070B5044641
:106C400025460DB1294600E00121084600F02CFF41
:106C5000002070BD10B500F055FF002010BD7FB5BD
:106C600004460D46606998B1A06988B1B4F908007E
:106C7000FFF7A6FF0646D4E90510CDE900610290B2
:106C80002B462269D4E9001001F090F8039013E03C
:106C9000B4F90800FFF794FF064603A8CDE90060A9
:106CA000238A9AB22B46D4E9001001F04DF801284E
:106CB00002D0002004B070BD0398FBE72DE9F0413D
:106CC00005460E461C4807681C480068001D00F079
:106CD000EFFD50B91948006890F82C100120884049
:106CE00017490968814316480160681C38B936B1F4
:106CF00012480168091D134800F024FE1AE07C19AF
:106D00000E4800684460BC4207D20C480168091D67
:106D10000D48006800F0FCFD0CE008480168091D02
:106D20000A48006800F0F4FD09480068844201D276
:106D300007480460BDE8F081E0050020CC05002094
:106D4000E40500201C4A0020D4050020D0050020C6
:106D5000FC05002010B5044600F000FE2348006842
:106D6000401C224908602248006840B9204804605D
:106D70000846006801280DD100F03AF90AE01D48E4
:106D8000006838B91A480068C06AE16A884201D8C8
:106D90001748046018480068401C1749086094F8B8
:106DA0002C100120884015490968084313490860E0
:106DB000E16A01EB8101124A02EB8100211D00F022
:106DC000C1FD00F0F5FD0B48006868B10848006897
:106DD000C06AE16A884207D24FF0805009490860D2
:106DE000BFF34F8FBFF36F8F10BD0000DC05002095
:106DF000CC050020E8050020F8050020E40500206F
:106E00004049002004ED00E010B516E000F0A6FDBA
:106E10000C48C068C468201D00F04AFD0A4800689C
:106E2000401E0949086009480068401E074908607B
:106E300000F0BEFD204600F00BF804480068002872
:106E4000E4D110BD084A0020DC050020D805002050
:106E500010B5044694F8510030B9206B00F0C6FD1F
:106E6000204600F0C3FD1AE094F85100012803D138
:106E7000204600F0BBFD12E094F85100022801D139
:106E8000012000E0002050B900BF502080F311889D
:106E9000BFF34F8FBFF36F8F00BF00BFFEE710BD82
:106EA00030B54FF44063174800F007042CB1C01D03
:106EB00020F00700134C041B1B1B0246124C2260DF
:106EC0000024114D6C60D018083820F007000F4CDA
:106ED000206000240D4D2D686C600C4D2D682C60D9
:106EE0001146441A4C60094C24680C60084D4C68EB
:106EF0002C60084D4C682C604FF00044064D2C600F
:106F000030BD0000304A0020080600201006002096
:106F100018060020140600201C06002000BFFFF702
:106F200073FF064800680128F9D94FF080500449E2
:106F30000860BFF34F8FBFF36F8FF0E74049002029
:106F400004ED00E02DE9FF5F81460F469246DDE942
:106F50000E6B109CAAF10100216B01EB800828F058
:106F6000070808F0070008B9012000E0002050B928
:106F700000BF502080F31188BFF34F8FBFF36F8F96
:106F800000BF00BFFEE7002507E0795D04F1340093
:106F90004155785D00B902E06D1C102DF5D300BF9E
:106FA000002143200155072E00D30626E6626664C1
:106FB0000020A064201D00F0A8FC04F1180000F0DF
:106FC000A4FC2461C6F10700A06164620020E064B3
:106FD00084F8500049464046039A00F049F9206081
:106FE000BBF1000F01D0CBF80040BDE8FF9F0000CF
:106FF00010B5002407E004EB84010F4A02EB810086
:1070000000F076FC641C072CF5D30C4800F070FCF3
:107010000B4800F06DFC0B4800F06AFC0A4800F0D9
:1070200067FC0A4800F064FC044809490860044809
:107030000849086010BD000040490020CC490020EC
:10704000E0490020F4490020084A00201C4A0020A2
:10705000D0050020D405002010B50146164800E0F8
:10706000006803688B42FBD30246436813448B429B
:1070700004D143684C682344436001460A464B6888
:1070800013440468A34211D10C4C03682468A34242
:1070900008D04B680468646823444B6003681B682D
:1070A0000B6005E0054B1B680B6001E003680B609B
:1070B000884200D0016010BD0806002010060020A4
:1070C0000A490968096809B9012100E0002121B1D4
:1070D0004FF0FF31064A116006E004490968C968AB
:1070E000C868034A4168116070470000D00500205D
:1070F000FC0500200E480068401C08B9012000E093
:10710000002050B900BF502080F31188BFF34F8F8B
:10711000BFF36F8F00BF00BFFEE700BF502080F3BA
:107120001188BFF34F8FBFF36F8F00BF00BFFEE723
:10713000200600202DE9F04104464FF0000800F041
:1071400039FD4648006808B9FFF7AAFE44480068C0
:10715000204000286BD1D4B1083404F00700B0B14E
:1071600004F00700C0F10800044404F0070008B967
:10717000012000E0002050B900BF502080F31188AA
:10718000BFF34F8FBFF36F8F00BF00BFFEE7002C30
:107190004DD034480068844249D8334E30460568A3
:1071A00001E02E462D686868A04202D228680028B7
:1071B000F7D12A480068854239D0306800F10808C4
:1071C000286830606868001B102819D92F1907F04B
:1071D000070008B9012000E0002050B900BF50208E
:1071E00080F31188BFF34F8FBFF36F8F00BF00BFD5
:1071F000FEE76868001B78606C603846FFF72CFF7C
:10720000184968680968081A16490860084600683D
:1072100016490968884203D2124800681349086079
:107220000F4968680968084368600020286000F01A
:10723000BDFE08F0070008B9012000E0002050B9A9
:1072400000BF502080F31188BFF34F8FBFF36F8FC3
:1072500000BF00BFFEE74046BDE8F08110060020F9
:107260001C06002014060020080600201806002036
:10727000001F4FF080730360001F21F001030360C3
:10728000001F034B03601438026020387047000071
:10729000F570000810B50548FCF714F84FF480624B
:1072A00003490248FCF744FB10BD0000784700206A
:1072B000CC36002002460948006838B1002002E0C0
:1072C0000B5C1354401C0528FADB06E0002002E0AA
:1072D0000B5C1354401C0428FADB70473400002078
:1072E000014608887047000010B504462046FFF7A5
:1072F000F7FF03464FF6FF70834204D1034800882E
:107300000249088001E00148038010BD720000209E
:107310002DE9FE4F06460F4690461D46DDE90C9AC4
:107320000E9C0020009001900290F0B28DF80000B9
:107330008DF801708DF8028028128DF80300E8B2F4
:107340008DF804004FEA29208DF8050009F0FF00B0
:107350008DF806004FEA2A208DF807000AF0FF009A
:107360008DF80800A01EC1B26846FFF737F98346C2
:107370000BF0FF01A01E0DF800104FEA2B21601E3C
:107380000DF80010631EA2B269460448FCF7EFFA3C
:10739000FFF75CF9FFF77EFFBDE8FE8F784700201E
:1073A0002DE9F04F85B006460F4690461D46DDE9B3
:1073B0000FABDDF83890119C0020019002900390F3
:1073C0000490F0B28DF804008DF805708DF80680F9
:1073D00028128DF80700E8B28DF808004FEA29203E
:1073E0008DF8090009F0FF008DF80A004FEA2A2005
:1073F0008DF80B000AF0FF008DF80C004FEA2B20EF
:107400008DF80D000BF0FF008DF80E00A01EC1B22C
:1074100001A8FFF7E3F800900098C1B2A01E01AAEE
:10742000115400980112601E1154631EA2B201A9EA
:107430000448FCF79CFAFFF709F9FFF72BFF05B0AA
:10744000BDE8F08F784700202DE9F04F85B0064663
:107450000F4690461D46DDE911B4DDE90E9A002085
:107460000190029003900490F0B28DF804008DF822
:1074700005708DF8068028128DF80700E8B28DF8A7
:1074800008004FEA29208DF8090009F0FF008DF867
:107490000A004FEA2A208DF80B000AF0FF008DF851
:1074A0000C00109800128DF80D001098C0B28DF8E5
:1074B0000E004FEA2B208DF80F000BF0FF008DF827
:1074C0001000A01EC1B201A8FFF788F80090009834
:1074D000C1B2A01E01AA115400980112601E1154DD
:1074E000631EA2B201A90548FCF741FAFFF7AEF806
:1074F000FFF7D0FE05B0BDE8F08F00007847002010
:107500002DE9FC4706460F4690461D460A9C002082
:1075100000900190F0B28DF800008DF801708DF8A8
:10752000028028128DF80300E8B28DF80400A01E36
:10753000C1B26846FFF752F8814609F0FF01A01E6C
:107540000DF800104FEA2921601E0DF80010A2B2BC
:10755000234669460448FCF70AFAFFF777F8FFF775
:1075600099FEBDE8FC870000784700202DE9FC412A
:107570000746884614461D46002000900190F8B248
:107580008DF800008DF8018020128DF80200E0B225
:107590008DF8030028128DF80400E8B28DF805007C
:1075A00006216846FFF71AF80646F0B28DF8060085
:1075B00030128DF807000723082269460448FCF7BB
:1075C000D6F9FFF743F8FFF765FEBDE8FC81000040
:1075D000784700202DE9FE4F06460F4690461D468F
:1075E000DDE90C940020009001900290F0B28DF83B
:1075F00000008DF801708DF8028028128DF80300CC
:10760000E8B28DF804004FEA29208DF8050009F052
:10761000FF008DF80600A01EC1B26846FEF7DEFF2F
:1076200082460AF0FF01A01E0DF800104FEA2A2141
:10763000601E0DF80010631EA2B269460448FCF7F4
:1076400096F9FFF703F8FFF725FEBDE8FE8F00006F
:10765000784700202DE9FE4306460F4614461D4696
:10766000DDF828900020009001900290F0B28DF893
:1076700000008DF8017020128DF80200E0B28DF844
:10768000030028128DF80400E8B28DF805008DF88B
:10769000069007216846FEF7A1FF804608F0FF002C
:1076A0008DF807004FEA28208DF8080009231A46B4
:1076B00069460448FCF75BF9FEF7C8FFFFF7EAFDEF
:1076C000BDE8FE837847002010B504464FF6FF70F2
:1076D000844214D1002208211548FAF7CFFD002278
:1076E00010211348FAF7CAFD002220211048FAF7AA
:1076F000C5FD002240210E48FAF7C0FD17E004F056
:10770000010208210A48FAF7B9FDC4F3400210212A
:107710000748FAF7B3FDC4F3800220210448FAF7C2
:10772000ADFDC4F3C00240210148FAF7A7FD10BD2A
:10773000000C014010B50446072C04DC074951F841
:107740002400FEF767FF4FF6FF70844201D0032C40
:1077500003D14FF41650FEF75DFF10BD5C0500200D
:1077600010B50446022221461648F9F7B5FA002062
:107770000FE0144931F810104FF47F4202EA012162
:10778000104A32F8102041EA12210E4A22F8101055
:10779000401C0128EDDB0B4800884FF6FF71884242
:1077A00003D10020084908600BE0064800884FF428
:1077B0007F4101EA00200349098840EA112002497B
:1077C000086010BD540500202800002038B504468C
:1077D000082212491248F9F77FFA00200FE01049F9
:1077E00031F810104FF47F4202EA01210C4A32F8BE
:1077F000102041EA12210A4A22F81010401C0428E5
:10780000EDDB69460648FEF73BFF0098401C00B9D7
:1078100038BD04490098086000BFF9E788F0070800
:10782000060000207800002010B5044604222146FE
:107830000548F9F751FA044840880349098840EAA5
:1078400001400249086010BD420000203C000020B9
:1078500010B504460222211D0348F9F73DFA0248FB
:1078600000880249088010BD46000020400000202A
:1078700010B5044610220C490C48F9F72DFA0020E7
:107880000FE00A4931F810104FF47F4202EA01215B
:10789000064A32F8102041EA1221044A22F8101058
:1078A000401C0828EDDB10BD00500708960600209C
:1078B00001460A69D1E901309860D1E901035860B5
:1078C0005068884201D188685060002008611068C3
:1078D000401E106010687047034B0360034B0B6041
:1078E0008023136070470000303000208430002077
:1078F00000F1080141604FF0FF31816000F10801A3
:10790000C160016100210160704700210161704781
:1079100010B502460B685C1C0CB9106907E002F157
:10792000080000E04068446824689C42FAD9446832
:107930004C604C68A160886041600A611468641CF6
:10794000146010BD42684A6093688B609368596008
:107950009160086103685B1C0360704700BF5020A2
:1079600080F31188BFF34F8FBFF36F8F00BF0E48B6
:107970000068401C0C49086008460068012812D1C4
:107980000A480068C0B208B9012000E0002050B9E0
:1079900000BF502080F31188BFF34F8FBFF36F8F6C
:1079A00000BF00BFFEE770472006002004ED00E0A6
:1079B0000D48006850B900BF502080F31188BFF314
:1079C0004F8FBFF36F8F00BF00BFFEE70648006810
:1079D000401E054908600846006820B9002080F371
:1079E000118800BF00BF70472006002070B5064612
:1079F0003546002E3FD0083D2C461F496068096877
:107A0000084008B1012000E0002050B900BF50201C
:107A100080F31188BFF34F8FBFF36F8F00BF00BF9C
:107A2000FEE7206808B9012000E0002050B900BF3F
:107A3000502080F31188BFF34F8FBFF36F8F00BFCB
:107A400000BFFEE70C4960680968084098B12068EB
:107A500088B90949606809688843606000F0AAF83D
:107A60000649606809680844044908602046FFF731
:107A7000F3FA00F09BFA70BD1C06002014060020EB
:107A800000204FF0E02108618861064800684FF44B
:107A90007A71B0FBF1F0401E4FF0E0214861072001
:107AA00008617047C805002070B504460025D4B1B0
:107AB0001248006808B9012000E0002050B900BF5A
:107AC000502080F31188BFF34F8FBFF36F8F00BF3B
:107AD00000BFFEE700F06EF800212046FFF7EEF849
:107AE00000F064FA05463DB94FF080500449086043
:107AF000BFF34F8FBFF36F8F70BD000004060020EF
:107B000004ED00E010B586B000200590049003AAB3
:107B100004A905A8FFF7E0FE0022DDE904101346E2
:107B2000CDE9002102901CA11D48039A00F03EF906
:107B30001C4908600846006808B1012400E00024E0
:107B4000012C15D100BF502080F31188BFF34F8F57
:107B5000BFF36F8F00BF4FF0FF3013490860012063
:107B60001249086000201249086000F071F810E026
:107B7000601C08B1012000E0002050B900BF502077
:107B800080F31188BFF34F8FBFF36F8F00BF00BF2B
:107B9000FEE706B010BD000049444C45000000005F
:107BA0001D6F000800060020FC050020E8050020ED
:107BB000E005002002480068401C01490860704749
:107BC000040600201D48006818B101201C49086007
:107BD00032E000201A4908601A480068B0FA80F0C4
:107BE000C0F11F0101EB8100174A52F8200008B1D3
:107BF000012000E0002050B900BF502080F3118820
:107C0000BFF34F8FBFF36F8F00BF00BFFEE701EBE5
:107C100081020D4B03EB820042685268426000F122
:107C200008024368934202D1426852684260426847
:107C3000D268064B1A6000BF70470000040600209F
:107C4000F0050020E405002040490020CC0500207C
:107C50001CB53849084600780190FF200A4610708C
:107C60000846007800909DF8000000F0F0009DF8B4
:107C70000020904201D1012000E0002050B900BF57
:107C8000502080F31188BFF34F8FBFF36F8F00BF79
:107C900000BFFEE79DF8000000F05000264A10707B
:107CA0000720264A106009E024480068401E234A45
:107CB00010609DF800004006000E00909DF8000046
:107CC00000F080008028EFD01C480068C0F1070059
:107CD000042801D1012000E0002050B900BF50204D
:107CE00080F31188BFF34F8FBFF36F8F00BF00BFCA
:107CF000FEE7124800680002104A10601046008833
:107D000000F4E06010600B4A019810700C480068A5
:107D100040F470000A4908600846006840F070406E
:107D20000860FFF7ADFE002006490860F8F71EFA6C
:107D300000201CBD00E400E02406002028060020EE
:107D400020ED00E0200600202DE9FF4F85B08046A1
:107D500089461746DDE912ABB800FFF7EBF9064696
:107D600056B15420FFF7E6F904460CB1266304E04F
:107D70003046FFF73BFE00E000248CB1002084F881
:107D80005100CDE900ABCDE902403A4649464046B4
:107D9000089BFFF7D7F82046FEF7DCFF012501E03E
:107DA0004FF0FF35284609B0BDE8F08F2DE9F04FC0
:107DB00085B00746884691469A46DDE90EB6109C86
:107DC0000EB1012000E0002050B900BF502080F328
:107DD0001188BFF34F8FBFF36F8F00BF00BFFEE767
:107DE0000CB1012000E0002050B900BF502080F30A
:107DF0001188BFF34F8FBFF36F8F00BF00BFFEE747
:107E0000542003900398542801D1012000E0002061
:107E100050B900BF502080F31188BFF34F8FBFF3DC
:107E20006F8F00BF00BFFEE7B4B1AEB125462C4650
:107E30002E63022085F85100002004A953464A46CB
:107E4000CDE900B1CDE9025041463846FFF77AF856
:107E50002846FEF77FFF01E000200490049805B05B
:107E6000BDE8F08F2DE9F0414FF00008444800686C
:107E7000002877D143480068451C4248056015BB7F
:107E800041480068006808B9012000E0002050B9AE
:107E900000BF502080F31188BFF34F8FBFF36F8F67
:107EA00000BF00BFFEE73848076838480068364919
:107EB00008603648076036480068401C344908604E
:107EC000FFF7FEF800BF3348006885423CD300BF8F
:107ED0002D480068006808B9012000E0002020B1AA
:107EE0004FF0FF302B4908602DE027480068C0683C
:107EF000C4686668B54202D22648066023E0201DA9
:107F0000FFF7D6FCA06A18B104F11800FFF7D0FC07
:107F100094F82C10012088401F49096808431E4925
:107F20000860E16A01EB81011C4A02EB8100211D1E
:107F3000FFF708FD1A49E06A0968C96A8842C7D391
:107F40004FF00108C4E700BF15480068C06A00EBA5
:107F50008000124951F82000012801D94FF0010892
:107F600005E0FFE70F480068401C0E4908600E4816
:107F7000006808B14FF001084046BDE8F0810000FC
:107F800004060020E0050020D0050020D4050020D4
:107F9000F4050020FC050020E405002040490020F5
:107FA000CC050020EC050020F005002070B5002471
:107FB00000263648006850B900BF502080F3118871
:107FC000BFF34F8FBFF36F8F00BF00BFFEE7FFF718
:107FD000C5FC2E480068401E2C4908600846006811
:107FE00000284FD12A48006800284BD024E02948B7
:107FF000C068C46804F11800FFF75AFC201DFFF7A1
:1080000057FC94F82C100120884023490968084344
:1080100021490860E16A01EB8101204A02EB8100FD
:10802000211DFFF78FFC1E49E06A0968C96A884272
:1080300002D301201B4908601648006808B90120D6
:1080400000E000200028D2D00CB1FFF739F8164824
:10805000056865B100BFFFF705FF10B101201149A8
:1080600008606D1E002DF6D100200F4908600D48F4
:10807000006838B1012630070C490860BFF34F8F04
:10808000BFF36F8FFFF794FC304670BD04060020ED
:10809000DC050020F4490020E405002040490020D0
:1080A000CC050020F0050020EC05002004ED00E0E8
:1080B000000801400100000000080140020000002B
:1080C0000008014004000000000801400800000012
:1080D00000080140100000000008014020000000DE
:1080E000000801404000000000080140800000003E
:1080F000C0810008195800080300000000000000BB
:108100008000000000000000000000009C810008CA
:108110003956000803000000000000008000000045
:108120000000000000000000A8810008855600083B
:1081300003000000000000008000000000000000BC
:1081400000000000B48100088F5600080300000002
:10815000000000008000000000000000000000009F
:1081600002030405060708090A0B0C0D0E0F101078
:10817000010202030405060708090A0B0C0D0E0F85
:1081800010100102000000000000000001020304C2
:108190000607080900000000010203046D7954611C
:1081A000736B3032000000006D795461736B3033B3
:1081B000000000006D795461736B303400000000E2
:1081C0006961705461736B00E88100080000002051
:1081D00034060000820700081C86000834060020D0
:1081E000FC550000806200080126034A040862C1B1
:1081F000042E0808232320C21A1C041A18041A1477
:10820000041A10041A0C041A08041A04041119049C
:108210001AF85D1AF0041AE8041AE0041AD8041ACD
:10822000D0041AC8041AC0041AB8041AB0041AA850
:10823000041AA0041A98041A90041A88041A8004D4
:108240001A70041A60041A50041A40041A30041AEE
:1082500020042A10B529541AC04819041AA0041A77
:1082600080041A400411290C62BF33803F1A400376
:1082700019041A80041AA0041AC0041AE004111A7E
:10828000414819041A20041A30041A40041A5004F0
:108290001A60041A70041A80041A88041A90041AC6
:1082A00098041AA0041AA8041AB0041AB8041AC030
:1082B000041AC8041AD0041AD8041AE0041AE804EC
:1082C0001AF0041AF8041122421A04041A08041AB3
:1082D0000C041A10041A14041A18041A1C041A2084
:1082E000041A24041A28041A2C041A30041A340418
:1082F0001A38041A3C041A40041A44041A48041A8E
:108300004C041A50041A54041A58041A5C041A60D3
:10831000041A64041A68041A6C041A70041A7404A7
:108320001A78041A7C041A80041A82041A84041A23
:1083300086041A88041A8A041A8C041A8E041A9065
:10834000041A92041A94041A96041A98041A9A04A5
:108350001A9C041A9E041AA0041AA2041AA4041A4D
:10836000A6041AA8041AAA041AAC041AAE041AB075
:10837000041AB2041AB4041AB6041AB8041ABA04D5
:108380001ABC041ABE041AC0041AC2041AC4041A7D
:10839000C6041AC8041ACA041ACC041ACE041AD085
:1083A0000400FF00D242CC76AA4348709F43EB32D0
:1083B000954324AF8B43A5D68243A13875433EE84D
:1083C000654318A65743D95D4A43E0FC3D43137209
:1083D0003243A5AD274313A11D43FA3E14430F7B3F
:1083E0000B43EF4903434142F742FAEDE8421F8550
:1083F000DB423FF7CE421835C3427D30B8426ADCDB
:10840000AD42E72CA442A1169B42428F9242438D7B
:108410008A42A107834271EC774282A26A425423C6
:108420005E42B16152424E514742B5E63C423F176F
:10843000334217D92942EB2221423DEC18420E2D3E
:10844000114201DE0942E9F7024210E9F841719B4D
:10845000EC41B3FBE0412EFFD541439CCB4186C9A3
:10846000C141917EB84133B3AF41D95FA741BF7DD0
:108470009F41F00598417CF29041713D8A41B1E104
:10848000834168B37B41F24170416666654159178B
:108490005B41D34D51410C0248410E2D3F414BC829
:1084A000364120099FCD2E414C37274110152041E0
:1084B00068221941029A12417C610C418E75064175
:1084C000B7D118F9418FE4F6401EA7EC408FE4E2E3
:1084D000405396D940AEB6D040143FC8406B2BC035
:1084E00040C976B840A01AB1407B14AA409E5EA352
:1084F00040C3F59C40D0D596407FFB9040B7628B3F
:1085000040D50986401CEB80401B0D78407DAE6E47
:108510004017B76540A3235D40EEEB5440B30C4DCC
:10852000404D8445408C4A3E40705F37400EBE301F
:10853000407C612A4017482440986E1E405BD31847
:10854000407671134045470E40835109408A8E049E
:108550004072F9FF3F9031F73F27C2EE3FA9A4E6F2
:108560003F5DDCDE3F705FD73FE02DD03F2041C94B
:108570003F3199C23FCA32BC3FA60AB63F7E1DB00A
:108580003F0A68AA3F4BEAA43FF9A09F3FCE889AD2
:108590003FCBA1953FA7E8903F1D5A8C3F72F987CA
:1085A0003F1AC0833F9B557F3FA779773F57EC6FBA
:1085B0003F029A683FC58F613F83C05A480033101D
:1085C000543F0DE04D3FBEC1473FDCD7413FF62849
:1085D0003C3FF0A7363FCA54313F11362C3FAB3EEB
:1085E000273F2575223FF2D21D3F1058193F8104C5
:1085F000153F5AFF01C123B00423600923C0123381
:108600008025324B329632E113C201024380321090
:0C8610004201035524F41AAA01011000D5
:0400000508000131BD
:00000001FF
